:020000040800F2
:10000000C8F300205D020008253B0008ED3500081C
:10001000213B000851070008295600080000000095
:100020000000000000000000000000009D0100082A
:10003000DB0B000800000000F9010008354A000849
:1000400077020008770200087702000877020008AC
:10005000770200087702000877020008770200089C
:10006000770200087702000877020008770200088C
:10007000B10A00087702000877020008770200083A
:10008000770200087702000877020008770200086C
:100090005507000877020008770200087702000879
:1000A000770200087702000877020008770200084C
:1000B000770200087702000877020008770200083C
:1000C000770200087702000877020008770200082C
:1000D000770200087155000877020008C95500082A
:1000E000770200087702000877020008770200080C
:1000F00077020008770200087702000877020008FC
:1001000077020008770200087702000877020008EB
:100110007702000877020008194B000877020008F0
:100120007702000877020008C10A00087702000879
:1001300077020008770200087702000877020008BB
:1001400065070008770200087702000877020008B8
:10015000770200087702000877020008770200089B
:10016000770200087702000877020008770200088B
:1001700077020008770200087702000800000000FC
:100180007702000877020008DFF80CD000F0BCFA14
:1001900000480047F15B0008C8F300202C4B1968A9
:1001A0000868B0E8F04F80F30988BFF36F8F4FF015
:1001B000000080F3118870470000000008480068C4
:1001C000006880F308884FF0000080F3148862B65E
:1001D00061B6BFF34F8FBFF36F8F00DF00BF00BF6B
:1001E00008ED00E0DFF80C00016841F470010160E7
:1001F000704700BF88ED00E0EFF30980BFF36F8F19
:10020000134B1A681EF0100F08BF20ED108A20E96A
:10021000F04F106009B44FF0500080F31188BFF325
:100220004F8FBFF36F8F06F0C1FF4FF0000080F3D8
:10023000118809BC19680868B0E8F04F1EF0100F6B
:1002400008BFB0EC108A80F30988BFF36F8F704746
:1002500048000020EFF30580704700000648804703
:1002600006480047FEE7FEE7FEE7FEE7FEE7FEE79B
:10027000FEE7FEE7FEE7FEE7054B00088901000800
:100280002DE9F05F0546002092469B4688460646CB
:10029000814640241BE0284641464746224600F05E
:1002A000B4F953465A46C01A914110D31146184624
:1002B000224600F09BF92D1A67EB01084F462246B3
:1002C0000120002100F092F917EB00094E41201E99
:1002D000A4F10104DFDC484631462A464346BDE826
:1002E000F09F40EA01039B0703D009E008C9121FF1
:1002F00008C0042AFAD203E011F8013B00F8013BE0
:10030000521EF9D27047D2B201E000F8012B491E0B
:10031000FBD270470022F6E710B513460A460446A2
:100320001946FFF7F0FF204610BD2DE9FE4F80462D
:1003300081EA0300C00F0C46009021F0004123F039
:100340000045B8EB0200A94105D24046214690463F
:100350001C460B46024623F00040104347D0270DB1
:10036000C7F30A00C3F30A510290401A01904028D3
:100370006BDAC3F3130040F4801B0098924620B15F
:100380000023D2EB030A63EB0B0B01985946C0F133
:100390004002504600F02AF906460D46504659469E
:1003A000019A00F042F910EB08006141002487EA4D
:1003B000115284EAE7731A4340D0009A62B3019A5B
:1003C000012A4FEA075215DC001B61EB02014FF0D6
:1003D000004202EA0752CDE90042001C41F58011BB
:1003E00032462B4600F042F903B0BDE8F08F40469C
:1003F0002146F9E7001B61EB0201001C41F5801367
:1004000000185B412018A2F5001747EB030140EAF2
:10041000D570B6196D4111E06D084FEA360645EA10
:10042000C0754FEA0752001B61EB0201001C41F549
:10043000801149084FEA30000019514132462B46DD
:1004400003B0BDE8F04F00F002B90098012240006F
:100450000023D0EB020263EBE073009821464FEAE1
:10046000E074B8EB000061EB0401E9E783F00043BE
:100470005BE781F0004158E72DE9FE4F81EA030474
:1004800004F0004421F0004100944FF0000B23F0F1
:10049000004350EA01045ED052EA03045BD0C3F388
:1004A0000A54C1F30A552C44A4F2F3340194A0FB7E
:1004B0000254C1F3130141F48011C3F3130343F455
:1004C000801301FB024400FB034E840A970A44EAAE
:1004D000815447EA8357A4FB076802958D0A05FB00
:1004E00007854FEA932C04FB0C542705029D4FEA25
:1004F000065847EA1637B5EB08056EEB070C870E72
:10050000920E47EA811742EA8312A7FB0201B6EB7B
:100510000B0164EB00042B0D43EA0C335E1844EB33
:100520001C50DA465146E7FB0201C5F313044FEABB
:100530000B3343EA14534FEA0432019C43EA0603A7
:10054000A4F10C040294009CCDE900B400F08EF8F4
:1005500003B0BDE8F08F00200146F9E70EB5C10FEA
:1005600080EAE0700844CA07002140F233438DE876
:100570000E000A460B4600F079F803B000BD70B5D6
:10058000C1F30A5201F000450024C1F3130140F207
:10059000FF3341F480119A4201DA002070BD40F22D
:1005A00033439A42A2F2334203DC524200F02DF868
:1005B00000E090402C43F1D0404270BD30B5041EA5
:1005C00071F1000404DB4FF00044404264EB010190
:1005D000141E73F1000405DB1C464FF00043524229
:1005E00063EB04038B4208BF824230BD202A04DB48
:1005F000203A00FA02F1002070479140C2F1200336
:1006000020FA03F3194390407047202A04DB203A74
:1006100021FA02F00021704721FA02F3D040C2F122
:1006200020029140084319467047202A06DBCB1769
:10063000203A41FA02F043EAE07306E041FA02F39D
:10064000D040C2F12002914008431946704710B5CE
:10065000141E73F1000408DA401C41F100019218E5
:100660005B411A4301D120F0010010BD2DE9F04D8E
:1006700092469B4611B1B1FA81F202E0B0FA80F2E3
:1006800020329046FFF7B2FF04460F4640EA0A00C8
:1006900041EA0B0153465A46084313D0114653EA28
:1006A000010019D0C8F140025046FFF7AEFF0546E1
:1006B0000E46504659464246FFF798FF084305D07C
:1006C000012004E020463946BDE8F08D00200543B6
:1006D00046EAE0762C4337430A986305E40AA0EB28
:1006E00008000022FD0A44EA47540A3002D50020DF
:1006F0000146E9E7010510196941DDE908450019DE
:100700006941BDE8F04DA2E7064C074D06E0E06800
:1007100040F0010394E8070098471034AC42F6D348
:10072000FFF736FD748100089481000810B500249D
:1007300008E08021054801F02BFB642001F01AFA43
:10074000601CC4B2042CF4DB10BD00000018024091
:1007500000BFFEE710B5024800F083FC10BD0000AA
:10076000C800002010B5024800F07BFC10BD00005E
:10077000F000002000B58BB0012009900020069009
:10078000059001900290039004900790012008903A
:100790000E200A9001A9154800F0E4FA08B100F013
:1007A0001DFA124800F065FF08B100F017FA0221A7
:1007B0000E4800F016FA08B100F010FA0E2006906C
:1007C00001A90B4800F0CEFA08B100F007FA08487A
:1007D00000F04FFF08B100F001FA0221044800F0D8
:1007E00000FA08B100F0FAF90BB000BDC800002013
:1007F000F000002070B506460C480088401C0B49EC
:1008000008804FF400710A4801F0C2FA06F016FDA4
:10081000054606F019FD0446044800884EF660219E
:10082000884202DB00200149088070BD00000020E2
:1008300000180240F0B585B006460C4617461D4626
:100840005FA103C9CDE903015DA103C9CDE90101A0
:10085000102E03D05C480088102854D15B480078E3
:1008600010B101284ED124E02F208DF80C008DF816
:10087000040000208DF80D008DF8050010208DF883
:1008800010008DF80800082003AB40F2016200213F
:1008900000904F4805F03CF9082001AB40F202629D
:1008A000002100904A4805F033F9012047490870BB
:1008B00028E02B208DF80C008DF8040001208DF825
:1008C0000D008DF8050000208DF810008DF808004F
:1008D0008DF811008DF80900082003AB40F2016289
:1008E000002100903A4805F013F9082001AB40F2CE
:1008F000026200210090364805F00AF900203349D1
:10090000087000BF5AE03348007810B1012854D174
:1009100027E02F208DF80C008DF8040000208DF8C2
:100920000D008DF805002C4800788DF81000264841
:1009300000788DF80800082003AB40F20162002126
:100940000090234805F0E4F8082001AB40F2026271
:10095000002100901E4805F0DBF801201D490870B9
:100960002BE02B208DF80C008DF8040001208DF871
:100970000D008DF80500E0B28DF81000E8B28DF89A
:100980000800200A8DF81100280A8DF809000820B7
:1009900003AB40F20162002100900D4805F0B8F869
:1009A000082001AB40F2026200210090084805F0E7
:1009B000AFF800200749087000BF00BF05B0F0BDC8
:1009C0002B00200010000000300000203400002028
:1009D000F0000020350000202E00002000B585B07A
:1009E0002FA003C8CDE903012DA103C9CDE9010161
:1009F0002D48007810B101284ED124E02F208DF829
:100A00000C008DF8040000208DF80D008DF8050015
:100A100010208DF810008DF80800082003AB40F27C
:100A2000016200210090214805F072F8082001AB16
:100A300040F20262002100901C4805F069F8012094
:100A40001949087028E02B208DF80C008DF804005F
:100A500001208DF80D008DF8050000208DF81000A4
:100A60008DF808008DF811008DF80900082003ABFF
:100A700040F20162002100900C4805F049F808207E
:100A800001AB40F2026200210090084805F040F8F6
:100A900000200549087000BF00BF05B000BD000080
:100AA0002B0020001000000034000020F000002087
:100AB00010B5024800F07EFE10BD000008090020BD
:100AC00010B5024800F076FE10BD0000A808002016
:100AD0000146087810381823B0FBF3F20848805C10
:100AE000C865032A05D908686FF30900001D8865E9
:100AF00003E008686FF309008865886D704700009F
:100B0000F0800008014600208A6A8B69CBB932B1B7
:100B1000012A0DD0022A03D0032A10D10EE000BF13
:100B2000CB6A03F08073B3F1807F00D1012007E02E
:100B3000CB6AB3F1C07F00D1012001E000E000BF2B
:100B400034E08B69B3F5005F1AD132B1012A07D0C6
:100B5000022A03D0032A11D10AE000BF01200EE0CF
:100B6000CB6A03F08073B3F1807F00D1012006E0EF
:100B7000CB6AB3F1C07F00D1012000E000BF15E0D7
:100B800032B1012A05D0022A04D0032A0CD103E095
:100B900000BF00BF012008E0CB6A03F08073B3F10F
:100BA000807F00D1012000E000BF00BF704730B55A
:100BB0000468246824F4802405682C600468636059
:100BC0008468402C04D10468A2600468E16003E0FA
:100BD0000468A1600468E26030BD704772B600BF6F
:100BE000FEE710B5024692F82030012B01D0022B0F
:100BF00006D110684069084314686061002010BD88
:100C0000506A40F4802050620120F8E7F0B50446B5
:100C10000D461E4694F8207020688368A86800B9C5
:100C200000E000BF012F01D0022F7CD103F08060D3
:100C300030B903F0006018B903F08050002873D079
:100C4000C3F30161022905D9606A40F400006062C3
:100C50000120F0BD012088403060A86860B9B5F877
:100C600000C0E86840EA4C5C206800F5C07000EB0A
:100C70000110C0F800C00FE0D5E901C040EACC0087
:100C8000D5F80CC040EA0C00D4F800C00CF5C07CCC
:100C90000CEB011CCCF80000D5F810C0206800F562
:100CA000C07000EB0110C0F804C0287D01280ED1EF
:100CB000206800F5C07000EB0110406840F4807CB3
:100CC000206800F5C07000EB0110C0F804C0D079B6
:100CD000000692F806C040EA0C4092F805C040EACF
:100CE0000C2C10794CEA000C206800F5C07000EB69
:100CF0000110C0F80CC0D078000692F802C040EA9B
:100D00000C4092F801C040EA0C2092F800C040EA82
:100D10000C00D4F800C00CF5C07C0CEB011CCCF826
:100D20000800206801E016E00FE000F5C07000EB5D
:100D30000110006840F0010C206800F5C07000EB65
:100D40000110C0F800C0002083E7606A40F4001082
:100D5000606201207DE7606A40F4802060620120CB
:100D600077E70000F0B504460A46216894F8205061
:100D7000012D01D0022D7ED1424901F50071086894
:100D800040F001000860086820F47C5008600868A2
:100D9000566A40EA06200860107D00F01F06012018
:100DA00000FA06F3C8699843C861A1F50071D069DB
:100DB000C8B9D1F80C029843C1F80C02908880B2EF
:100DC000968940EA064601F51070576940F8376089
:100DD000108880B2168940EA064601F510705769FE
:100DE00000EBC7004660D069012819D1D1F80C0288
:100DF0001843C1F80C02908880B2168840EA064673
:100E000001F51070576940F83760908980B21689F3
:100E100040EA064601F51070576900EBC7004660CE
:100E2000906928B9D1F804029843C1F8040204E09B
:100E3000D1F804021843C1F80402106928B9D1F8A6
:100E400014029843C1F8140204E0D1F814021843C4
:100E5000C1F81402106A012804D1D1F81C02184309
:100E6000C1F81C02D1F8000220F00100C1F8000214
:100E70000020F0BDFFE7606A40F48020606201203E
:100E8000F7E7000000640040704710B502460020FC
:100E900092F82030012B01D0022B09D121B914681E
:100EA000E46804F0030003E01468246904F003001C
:100EB00010BD70B5044694F82050012D01D0022DCC
:100EC0007DD151B92068C06800F0030080B9606A24
:100ED00040F400106062012070BD2068006900F0DD
:100EE000030028B9606A40F4001060620120F3E753
:100EF000206800F5D87000EB0110006800F00400D5
:100F00009060906840B9206800F5D87000EB01103F
:100F10000068400D106007E0206800F5D87000EB15
:100F200001100068C0085060206800F5D87000EB20
:100F30000110006800F00200D060206800F5D87051
:100F400000EB0110406800F00F001061206800F510
:100F5000D87000EB0110406800F47F40000A9061F7
:100F6000206800F5D87000EB01104068000C50615B
:100F7000206800F5D87000EB0110806818702068B8
:100F800000F5D87000EB0110806800F47F40000A83
:100F90005870206800F5D87000EB0110806800F4EC
:100FA0007F00000C9870206800F5D87000EB0110ED
:100FB0008068000ED870206800F5D87000E02FE03F
:100FC00000EB0110C0681871206800F5D87000EBC4
:100FD0000110C06800F47F40000A5871206800F5D5
:100FE000D87000EB0110C06800F47F00000C98710D
:100FF000206800F5D87000EB0110C068000ED871B1
:1010000031B92068C06840F020002668F06005E033
:101010002068006940F020002668306100205BE70E
:10102000606A40F480206062012055E7014600209C
:1010300091F82020012A01D0022A11D10B689B6867
:1010400003F0806303B1401C0B689B6803F00063EE
:1010500003B1401C0B689B6803F0805303B1401C34
:1010600070472DE9F05F0446002520684669206836
:10107000D0F80490206887682068D0F80CA0206819
:10108000D0F810B02068D0F8188006F001000028D1
:1010900055D007F00100C0B101202168886007F039
:1010A000020018B1204600F014FB0EE007F0040027
:1010B00010B145F4006508E007F0080010B145F4F0
:1010C000805502E0204600F003FB07F48070C8B1B1
:1010D0004FF480702168886007F4007018B12046D2
:1010E00000F0F9FA0EE007F4806010B145F4005505
:1010F00008E007F4006010B145F4804502E02046A6
:1011000000F0E8FA07F48030C8B14FF4803021686D
:10111000886007F4003018B1204600F0DEFA0EE0D7
:1011200007F4802010B145F4004508E007F40020E2
:1011300010B145F4803502E0204600F0CDFA06F00B
:10114000080038B10AF0100020B145F400751020F5
:101150002168C86006F0040040B10AF0080028B118
:1011600008202168C860204600F00EFA06F0020050
:1011700038B12068C06800F0030010B1204600F0CC
:1011800005FA06F0400038B10BF0100020B145F42C
:10119000806510202168086106F0200040B10BF046
:1011A000080028B1082021680861204600F05EFA96
:1011B00006F0100038B12068006900F0030010B19B
:1011C000204600F054FA06F4003040B109F0100057
:1011D00028B1102021684860204600F049FA06F442
:1011E000803040B109F0080028B10820216848602B
:1011F000204600F073FA06F4004088B309F00400BA
:1012000078B306F4807020B108F0010008B145F011
:10121000010506F4007020B108F0020008B145F0A5
:10122000020506F4806020B108F0040008B145F022
:10123000040506F40060A0B108F0700088B108F061
:101240007000402817D006DC10280BD020280CD0C6
:10125000302819D10CE0502810D0602814D110E0AB
:101260001DE019E045F008050FE045F010050CE021
:1012700045F0200509E045F0400506E045F0800511
:1012800003E045F4807500E000BF00BF206880697E
:1012900020F07000216888610420216848602DB129
:1012A000606A284360622046FFF7EEFDBDE8F09FCC
:1012B00070B504460CB9012070BD94F8200010B937
:1012C000204600F0AFF82068006840F00100216877
:1012D000086000F06DFD05460DE000F069FD401B63
:1012E0000A2808D9606A40F400306062052084F85A
:1012F00020000120E0E72068406800F0010000289D
:10130000EBD02068006820F002002168086000F03F
:101310004FFD05460DE000F04BFD401B0A2808D9A3
:10132000606A40F400306062052084F820000120EB
:10133000C2E72068406800F002000028EBD1207E60
:10134000012806D12068006840F08000216808600C
:1013500005E02068006820F0800021680860607E59
:10136000012806D12068006840F04000216808602C
:1013700005E02068006820F0400021680860A07E39
:10138000012806D12068006840F02000216808602C
:1013900005E02068006820F0200021680860E07EF9
:1013A000012806D12068006820F01000216808603C
:1013B00005E02068006840F0100021680860207F88
:1013C000012806D12068006840F008002168086004
:1013D00005E02068006820F0080021680860607F50
:1013E000012806D12068006840F0040021680860E8
:1013F00005E02068006820F0040021680860D4E956
:101400000201084321690843616908436168491E74
:1014100008432168C86100206062012084F8200030
:10142000002049E710B586B00446142101A8FEF754
:1014300071FF4F492068884242D14E480068401CE5
:101440004C4908600846006801280FD100BF002001
:1014500000904948006840F000704749086008461D
:10146000006800F00070009000BF00BF00BF0020C7
:10147000009041481038006840F001003E491039A2
:1014800008600846006800F00100009000BF00BF3F
:101490004FF4C050019002200290002003900320DE
:1014A00004900920059001A9344800F077FB002240
:1014B0000521142000F048FD142000F035FD55E012
:1014C0002F492068884251D100BF002000902A484F
:1014D000006840F08060284908600846006800F015
:1014E0008060009000BF00BF22480068401C214976
:1014F00008600846006801280FD100BF0020009056
:101500001D48006840F000701B49086008460068EC
:1015100000F00070009000BF00BF00BF00200090EE
:1015200015481038006840F002001349103908606F
:101530000846006800F00200009000BF00BF4FF4B2
:10154000405001900220029000200390032004905C
:101550000920059001A90B4800F020FB002205217D
:10156000402000F0F1FC402000F0DEFC06B010BD91
:101570000064004014000020403802400000024097
:1015800000680040000402407047000010B598B0A9
:10159000044600200290039000212046FFF775FCCE
:1015A0002F4920680968884205D116AB0FAA00218F
:1015B0002046FFF77EFC2B492068096888424CD101
:1015C0000DAB06AA00212046FFF773FC40F28251C2
:1015D000069888421ED1DDE90D01CDE904019DF890
:1015E00010004B2839D19DF81200212835D19DF8E3
:1015F0001300022831D19DF8140040B28DF8040088
:101600009DF8150040B28DF80500BDF8041016488D
:10161000418122E040F28151069888421DD1DDE9E6
:101620000D01CDE902019DF808004B2815D19DF868
:101630000A00212811D19DF80B0001280DD19DF839
:101640000C0040B28DF804009DF80D0040B28DF8FA
:101650000500BDF804000449088118B010BD000061
:10166000C8000020F00000202810002070477047BC
:10167000704770B5044694F82000012822D102205A
:1016800084F820002068006820F0010021680860CC
:1016900000F08EFB05460DE000F08AFB401B0A2897
:1016A00008D9606A40F400306062052084F82000A8
:1016B000012070BD2068406800F001000028EBD1D7
:1016C0006062F6E7606A40F4002060620120F0E7A3
:1016D000704770477047704770477047704770B5E4
:1016E0000446A56D00F064FB064694F83500022818
:1016F00008D08020606500BF002084F8340000BF5F
:10170000012070BD2068006820F016002168086084
:101710002068406920F0800021684861206C08B989
:10172000A06C28B12068006820F0080021680860DB
:101730002068006820F001002168086010E000F0D7
:1017400037FB801B05280BD920206065032084F817
:10175000350000BF002084F8340000BF0320D0E72C
:101760002068006800F001000028E8D194F85C10BF
:101770003F208840A860012084F8350000BF002089
:1017800084F8340000BF00BFBBE7014691F8350084
:10179000022803D08020486501207047052081F889
:1017A00035000868006820F001000A681060002019
:1017B000F3E70000F8B50446002000908C4800686C
:1017C0004FF41651B0FBF1F7A56D2E6894F85C103C
:1017D00008208840304098B12068006800F004007C
:1017E00070B12068006820F004002168086094F857
:1017F0005C1008208840A860606D40F001006065C2
:1018000094F85C1001208840304068B1206840693D
:1018100000F0800040B194F85C1001208840A8607E
:10182000606D40F00200606594F85C100420884010
:10183000304068B12068006800F0020040B194F8C0
:101840005C1004208840A860606D40F00400606572
:1018500094F85C1010208840304078B3206800680D
:1018600000F0080050B394F85C1010208840A86085
:101870002068006800F4802080B12068006800F4CF
:10188000002028B9206CC8B12046216C884715E09B
:10189000A06C98B12046A16C88470FE020680068D2
:1018A00000F4807028B92068006820F008002168E2
:1018B0000860206C10B12046216C884794F85C10B9
:1018C000202088403040002865D02068006800F063
:1018D000100000285FD094F85C1020208840A86099
:1018E00094F83500052828D12068006820F01600FB
:1018F000216808602068406920F080002168486104
:10190000206C08B9A06C28B12068006820F008009D
:101910002168086094F85C103F208840A86001208E
:1019200084F8350000BF002084F8340000BF206D2B
:1019300010B12046216D8847F8BD2068006800F48A
:10194000802080B12068006800F4002028B9606C15
:1019500010B12046616C88471DE0E06BD8B120468D
:10196000E16B884717E02068006800F4807068B970
:101970002068006820F0100021680860012084F8C9
:10198000350000BF002084F8340000BFE06B10B1C8
:101990002046E16B8847606D38B3606D00F0010050
:1019A000F0B1052084F835002068006820F00100BF
:1019B0002168086000BF0098401C0090B84200D920
:1019C00005E02068006800F001000028F3D100BFA6
:1019D000012084F8350000BF002084F8340000BFE7
:1019E000E06C10B12046E16C884700BFA4E700001E
:1019F000440000202DE9F0410446002500F0D8F90C
:101A0000074614B90120BDE8F081606A00B100BF4B
:101A1000022084F8350000BF002084F8340000BFA5
:101A20002068006820F00100216808600AE000F0EA
:101A3000BFF9C01B052805D920206065032084F864
:101A40003500E0E72068006800F001000028EED1D2
:101A50002068056821480540D4E901010843E16890
:101A600008432169084361690843A1690843E169A2
:101A70000843216A08430543606A042803D1D4E976
:101A80000B0108430543206805602068456925F07F
:101A90000705606A0543606A04280DD1A06A054302
:101AA000E06A48B12046FFF72DF828B14020606574
:101AB000012084F83500A6E7206845612046FFF73D
:101AC00007F8064694F85C103F208840B06000207C
:101AD0006065012084F83500002094E73F8010F015
:101AE0002DE9F04704460D4616461F464FF0000804
:101AF000D4F8589000BF94F83400012802D1022095
:101B0000BDE8F087012084F8340000BF94F8350068
:101B1000012825D1022084F83500002060653B466D
:101B2000324629462046FFF742F894F85C103F20E1
:101B30008840C9F808002068006840F01600216855
:101B40000860206C28B12068006840F00800216817
:101B500008602068006840F001002168086006E025
:101B600000BF002084F8340000BF4FF00208404658
:101B7000C6E7000070B5044600F01AF9064625468F
:101B8000681C10B104480078054400BF00F010F94B
:101B9000801BA842FAD370BD40000020F8B5024671
:101BA0000B460025002400200021D6E0012606FA7D
:101BB00001F51E6806EA0504AC4274D11E7906F0F0
:101BC0000306012E04D01E7906F00306022E13D15F
:101BD00090684F000326BE40B0434F00DE68BE4011
:101BE00030439060506801268E40B0431E79C6F3A2
:101BF00000168E40304350601E7906F00306032E17
:101C000009D0D0684F000326BE40B0434F009E6805
:101C1000BE403043D0601E7906F00306022E13D179
:101C2000CF0802F1200656F827004E07F70E0F26C0
:101C3000BE40B0434F07FF0E1E69BE403043CF0881
:101C400002F1200646F8270010684F000326BE4028
:101C5000B0431E7906F003064F00BE4030431060CB
:101C60005E6806F44036002E76D000BF002600964F
:101C70003C4E366846F480463A4F3E603E463668F3
:101C800006F48046009600BF00BF374E8F0856F816
:101C900027008E07370F0F26BE40B043334EB242A7
:101CA00002D1002624E057E0314EB24201D1012694
:101CB0001EE0304EB24201D1022619E02E4EB24251
:101CC00001D1032614E02D4EB24201D104260FE0CB
:101CD0002B4EB24201D105260AE02A4EB24201D172
:101CE000062605E0284EB24201D1072600E008266C
:101CF0008F073F0FBE4030431B4E8F0846F827002A
:101D0000224E3068A0435E6806F4801606B1204378
:101D10001E4E3060361D3068A0435E6806F4001623
:101D200006B12043194E361D3060184E361F3068FC
:101D3000A0435E6806F4003606B12043134E361FFA
:101D40003060361F3068A0435E6806F4803606B106
:101D500020430E4E083E3060491C1029FFF426AF88
:101D6000F8BD00004438024008380140000002403D
:101D70000004024000080240000C02400010024033
:101D80000014024000180240001C0240083C0140C0
:101D900010B5426921EA020302EA010443EA04435E
:101DA000836110BD0AB1816101E00B04836170475A
:101DB00001480068704700003800002001464AF6DC
:101DC000AA200A68106000207047000003480068DD
:101DD0000349097808440149086070473800002029
:101DE0004000002010B50D48006840F400700B4919
:101DF00008600846006840F4806008600846006893
:101E000040F480700860032000F0DCF80F2000F040
:101E100007F800F05FF8002010BD0000003C024011
:101E20002DE9F04188B004460027B84600BF0020E5
:101E300001902348006840F01000214908600846DE
:101E4000006800F01000019000BF00BF02A903A8C5
:101E500000F08EF9069F1FB900F0B2F9054602E0C6
:101E600000F0AEF945001748B5FBF0F0A0F101080D
:101E700015481649086040F2E7311448C160C0F8BF
:101E80000480002101618160816100F0BBFC064695
:101E900096B90E4800F01CFD06466EB9362000F0DB
:101EA00043F8102C07D200222146362000F04CF8CF
:101EB0000748046000E00126304608B0BDE8F08124
:101EC0004038024040420F000010004068090020E6
:101ED0003C00002008B500BF0020009011480068B9
:101EE00040F480400F4908600846006800F48040D4
:101EF000009000BF00BF00BF00200090081F0068D6
:101F000040F08050091F08600846006800F08050CB
:101F1000009000BF00BF00220F21901E00F014F8B7
:101F200008BD00004438024001460846002809DB8D
:101F300000F01F0301229A4043099B0003F1E023B4
:101F4000C3F8002100BF70472DE9F05F80460D46C1
:101F50001646002703F0AEFD074639462A463346AB
:101F600001F00700C0F1070ABAF1040F02D94FF0DF
:101F7000040A01E0C0F1070AD14600F1040ABAF1EF
:101F8000070F02D24FF0000A01E0A0F1030AD44685
:101F90004FF0010A0AFA09FAAAF1010A0AEA020A4A
:101FA0000AFA0CFA4FF0010B0BFA0CFBABF1010B28
:101FB0000BEA030B4AEA0B042146404603F082FD7C
:101FC000BDE8F09F00BF00F00702064B19684FF60E
:101FD000FF031940044B0B4343EA0221014B1960F4
:101FE00000BF70470CED00E00000FA0570B5044634
:101FF0000D460CB9012070BD5848006800F007007C
:10200000A84209D255490D700846006800F0070043
:10201000A84201D00120EEE7207800F0020002285B
:102020001DD1207800F00400042805D14C48006838
:1020300040F4E0504A490860207800F00800082881
:1020400005D14748006840F460404549086044486D
:10205000006820F0F000A16808434149086020783A
:1020600000F00100A8B36068012807D13C48083897
:102070000068C0F34040B8B90120BCE7606802289E
:1020800002D06068032807D1354808380068C0F3DB
:10209000406048B90120AEE7314808380068C0F315
:1020A000400008B90120A6E72D48006820F0030091
:1020B000616808432A490860FFF77AFE064609E08E
:1020C000FFF776FE801B41F28831884202D9032057
:1020D00091E707E02248006800F00C006168B0EB6F
:1020E000810FEDD11D48006800F00700A84209D912
:1020F0001A490D700846006800F00700A84201D098
:10210000012078E7207800F00400042807D1144863
:10211000006820F4E050E168084311490860207825
:1021200000F00800082808D10D48006820F460403D
:10213000216940EAC1000A49086000F061F80849D5
:102140000968C1F30311074A515CC8400649086099
:1021500006480068FFF764FE00204CE7003C0240A0
:1021600008380240F8800008440000203C000020AD
:102170000F2202600D4A126802F0030242600B4A0D
:10218000126802F0F0028260084A126802F4E0521B
:10219000C260064A126802F46042D2080261044A30
:1021A000126802F007020A60704700000838024017
:1021B000003C0240014800687047000044000020D5
:1021C00000B5FFF7F7FF04490968C1F38221034A0C
:1021D000515CC84000BD000008380240088100087A
:1021E00000B5FFF7E7FF04490968C1F34231034A2C
:1021F000515CC84000BD000008380240088100085A
:102200002DE9F047002400250026A1462548006856
:1022100000F00C0020B1042805D008283AD105E0D0
:10222000DFF8849039E0DFF8849036E01D48001F25
:10223000006800F03F041B48001F006800F48000A5
:1022400078B11A481749091F0968C1F38811A0FB22
:1022500001700146224600233846FEF711F8054674
:102260000EE011480F49091F0968C1F38811A0FB4E
:1022700001700146224600233846FEF701F8054664
:102280000848001F0068C0F30140401C4600B5FB31
:10229000F6F902E0DFF8109000BF00BF4846BDE845
:1022A000F0870000083802400024F40000127A0091
:1022B000F8B504460CB90120F8BD207800F0010003
:1022C000002874D0F948006800F00C0004280DD0F4
:1022D000F648006800F00C00082813D1F348001FEE
:1022E000006800F48000B0F5800F0BD1EF4808388B
:1022F0000068C0F34040002859D06068002856D1DB
:102300000120D9E700BF6068B0F5803F08D1E748F9
:102310000838006840F48030E449083908601EE05D
:102320006068B0F5A02F0DD1E0480838006840F48F
:102330008020DE49083908600846006840F4803093
:1023400008600CE0D9480838006820F48030D7498C
:10235000083908600846006820F48020086000BF43
:10236000606890B1FFF724FD054606E0FFF720FD09
:10237000401B642801D903209EE7CC480838006838
:10238000C0F340400028F1D011E0FFF711FD0546F1
:1023900006E0FFF70DFD401B642801D903208BE701
:1023A000C24808380068C0F340400028F1D12078C6
:1023B00000F0020002285FD1BC48006800F00C0069
:1023C00058B1BA48006800F00C0008281CD1B74882
:1023D000001F006800F48000B0B9B44808380068F5
:1023E000C0F3400020B1E068012801D0012063E77C
:1023F000AE480838006820F0F800216940EAC100C2
:10240000AA490839086037E0E06800B30120A8490C
:102410000860FFF7CDFC054606E0FFF7C9FC401B4E
:10242000022801D9032047E7A04808380068C0F314
:1024300040000028F1D09D480838006820F0F800DE
:10244000216940EAC10099490839086014E0002078
:1024500097490860FFF7ACFC054606E0FFF7A8FCCB
:10246000401B022801D9032026E79048083800685D
:10247000C0F340000028F1D1207800F008000828BF
:102480002CD16069A8B101208A490860FFF790FC4F
:10249000054606E0FFF78CFC401B022801D903200B
:1024A0000AE782486C300068C0F340000028F1D091
:1024B00014E000207F490860FFF77AFC054606E03B
:1024C000FFF776FC401B022801D90320F4E6774889
:1024D0006C300068C0F340000028F1D1207800F093
:1024E0000400042870D1002770483830006800F0DC
:1024F000805090B900BF002000906C4838300068D0
:1025000040F080506949383108600846006800F0A2
:102510008050009000BF00BF01276748006800F4AA
:102520008070B0B96448006840F480706249086007
:10253000FFF73EFC054606E0FFF73AFC401B022889
:1025400001D90320B8E65C48006800F480700028D8
:10255000F2D000BFA068012808D154486830006854
:1025600040F001005149683108601DE0A06805286D
:102570000DD14E486830006840F004004B49683186
:1025800008600846006840F0010008600CE0474819
:102590006830006820F0010044496831086008464E
:1025A000006820F00400086000BFA068A8B1FFF731
:1025B000FFFB054609E0FFF7FBFB401B41F28831BA
:1025C000884202D9032077E626E038486830006860
:1025D000C0F340000028EED013E0FFF7E9FB05460A
:1025E00008E0FFF7E5FB401B41F28831884201D942
:1025F000032061E62D4868300068C0F340000028E1
:10260000EFD1012F07D129483830006820F08050E1
:1026100026493831086000BFA069002845D023480A
:10262000006800F00C0008285DD0A069022845D1A0
:1026300000201F490866FFF7BBFB054606E0FFF7D1
:10264000B7FB401B022801D9032035E6174808389C
:102650000068C0F340600028F1D1D4E907010843C5
:10266000616A40EA81110122A06AC2EB500041EA8E
:1026700000412C20005D41EA00600C49091F086000
:1026800001200B490866FFF793FB054606E0FFF7BC
:102690008FFB401B022801D903200DE603480838B0
:1026A0000068C0F340600028F1D049E008380240DB
:1026B00000004742800E4742007000400020214940
:1026C0000866FFF775FB054606E0FFF771FB401B48
:1026D000022801D90320EFE51B480068C0F34060E1
:1026E0000028F2D12CE0A069012800D1E4E51648C9
:1026F000001D0668A069012820D006F48001E06969
:1027000081421BD106F03F01206A814216D147F673
:10271000C0703040616AB0EB811F0FD106F44031C8
:102720000122A06AC2EB5000B1EB004F06D106F0C7
:1027300070612C20005DB1EB006F01D00120BBE582
:102740000020B9E50000474200380240704770475A
:1027500030B502460B4600BF92F83C00012801D17B
:10276000022030BD012082F83C0000BF022082F828
:102770003D00106844681068816824F0700418688F
:10278000044310684460184D1068A8421BD01068BC
:10279000B0F1804F17D0154D1068A84213D0144DDA
:1027A0001068A8420FD0134D1068A8420BD0124DEC
:1027B0001068A84207D0114D1068A84203D0104DF0
:1027C0001068A84205D121F08001586801431068C3
:1027D0008160012082F83D0000BF002082F83C00AB
:1027E00000BF00BFBDE70000000001400004004042
:1027F00000080040000C004000040140004001407F
:102800000018004010B504460CB9012010BD94F822
:102810003D0028B9002084F83C00204600F026F84E
:10282000022084F83D00211D206802F07DF901207E
:1028300084F8460000BF84F83E0001213F20015586
:10284000402001554120015500BF00BF012084F800
:10285000420043200155442001554520015500BF49
:10286000012084F83D000020D0E7000008B5154A9B
:10287000016891420FD100BF0021009112490968FF
:1028800041F00401104A11601146096801F0040189
:10289000009100BF15E00D4A0168914211D100BFBF
:1028A000002100910849091D096841F48031064A58
:1028B000121D11601146096801F48031009100BFBA
:1028C00000BF08BD00080040403802400040014001
:1028D000014691F83D00012801D0012070470220F7
:1028E00081F83D000868C06840F001000B68D860BE
:1028F0001A4B086898421BD00868B0F1804F17D077
:10290000174B0868984213D0164B086898420FD0AE
:10291000154B086898420BD0144B0868984207D0B2
:10292000134B0868984203D0124B086898420CD1A8
:102930000868806800F00702062A0CD00868006862
:1029400040F001000B68186005E00868006840F07E
:1029500001000B6818600020C0E700000000014083
:102960000004004000080040000C0040000401404A
:1029700000400140001800402DE9F04104460D469A
:10298000002700BF94F83C00012802D10220BDE8D6
:10299000F081012084F83C0000BF022084F83D0053
:1029A0002068866826F0770626F47F4620688660D1
:1029B0002868502833D00CDC202850D004DC0028B4
:1029C0004BD0102851D149E0302849D040284CD173
:1029D00039E060282DD0702807D0B0F5805F03D093
:1029E000B0F5005F41D10DE041E0D5E902136A681E
:1029F000206802F016F92068866846F0770620689D
:102A0000866034E0D5E902136A68206802F009F9AB
:102A10002068806840F480402168886027E0EA6888
:102A20006968206802F0EEF95021206802F004F98C
:102A30001DE0EA686968206802F0F7F96021206803
:102A400002F0FAF813E0EA686968206802F0DAF93F
:102A50004021206802F0F0F809E000BF00BF00BF8D
:102A60002968206802F0E8F801E0012700BF00BFF4
:102A7000012084F83D0000BF002084F83C0000BF26
:102A8000384684E7704710B5044620680069C0F3F3
:102A90004000D8B12068C068C0F34000B0B16FF00A
:102AA000020021680861012020772068806900F019
:102AB000030018B12046FFF7E5FF05E0204600F0CF
:102AC00029F9204600F0F6F90020207720680069F7
:102AD000C0F38000D8B12068C068C0F38000B0B1F6
:102AE0006FF0040021680861022020772068806967
:102AF00000F4407018B12046FFF7C4FF05E02046FF
:102B000000F008F9204600F0D5F900202077206871
:102B10000069C0F3C000D8B12068C068C0F3C0002D
:102B2000B0B16FF0080021680861042020772068A8
:102B3000C06900F0030018B12046FFF7A3FF05E0CD
:102B4000204600F0E7F8204600F0B4F90020207796
:102B500020680069C0F30010D8B12068C068C0F3D5
:102B60000010B0B16FF010002168086108202077D4
:102B70002068C06900F4407018B12046FFF782FF5A
:102B800005E0204600F0C6F8204600F093F900204A
:102B900020772068006900F0010058B12068C06803
:102BA00000F0010030B16FF001002168086120469B
:102BB00000F008FA20680069C0F3C01058B120681E
:102BC000C068C0F3C01030B16FF0800021680861A8
:102BD0002046FFF7BBFD20680069C0F3801058B1A4
:102BE0002068C068C0F3801030B16FF040002168E9
:102BF0000861204600F00CFA20680069C0F340101C
:102C000058B12068C068C0F3401030B16FF02000A8
:102C1000216808612046FFF79AFD10BD10B586B007
:102C20000446142101A8FDF775FB3349206888424A
:102C30001CD100BF002000903048006840F0020026
:102C40002E4908600846006800F00200009000BFAE
:102C500000BF022001900290002003900490022007
:102C6000059001A92648FEF799FF43E02549206811
:102C700088421ED100BF002000902048006840F02C
:102C800008001E4908600846006800F0080000902F
:102C900000BF00BF4FF4704001900220029000205E
:102CA000039004900220059001A91748FEF776FFD3
:102CB00020E01649206888421CD100BF0020009007
:102CC0000E48006840F010000C4908600846006893
:102CD00000F01000009000BF00BF602001900220B3
:102CE00002900020039004900320059001A9084859
:102CF000FEF754FF06B010BD00040040303802401B
:102D00000004024000080040000C02400040014066
:102D10000010024070472DE9F04104460D4616466A
:102D2000002700BF94F83C00012802D10220BDE832
:102D3000F081012084F83C0000BF36B1042E1BD086
:102D4000082E31D00C2E5ED145E02946206801F0D6
:102D50007DFF2068806940F0080021688861206854
:102D6000806920F0040021688861206880692969F1
:102D700008432168886148E02946206801F09EFFE9
:102D80002068806940F4006021688861206880695B
:102D900020F480602168886120688069296940EAA0
:102DA00001202168886130E02946206801F0C4FFD5
:102DB0002068C06940F008002168C8612068C069C7
:102DC00020F004002168C8612068C06929690843AF
:102DD0002168C86119E02946206801F0E9FF2068F0
:102DE000C06940F400602168C8612068C06920F4AF
:102DF00080602168C8612068C069296940EA0120B3
:102E00002168C86101E0012700BF00BF00BF0020AA
:102E100084F83C0000BF384689E710B504460CB979
:102E2000012010BD94F83D0028B9002084F83C0032
:102E3000204600F025F8022084F83D00211D20687E
:102E400001F072FE012084F8460000BF84F83E00C5
:102E500001213F200155402001554120015500BF6F
:102E600000BF012084F84200432001554420015551
:102E70004520015500BF012084F83D000020D0E727
:102E800008B50A4A016891420FD100BF00210091A4
:102E90000749096841F00201054A116011460968B5
:102EA00001F00201009100BF00BF08BD0004004016
:102EB000403802407047000070B504460D4615B911
:102EC00094F83E000BE0042D02D13F20005D06E0A7
:102ED000082D02D14020005D01E04120005D012865
:102EE00001D0012070BD1DB9022084F83E000EE023
:102EF000042D03D102213F20015508E0082D03D104
:102F000002214020015502E0022141200155012209
:102F10002946206801F074FE23492068884203D0C6
:102F200022492068884201D1012000E0002028B118
:102F30002068406C40F40040216848641A492068C9
:102F400088421BD02068B0F1804F17D01849206804
:102F5000884213D01749206888420FD0164920684C
:102F600088420BD011492068884207D01349206855
:102F7000884203D01249206888420CD120688068BA
:102F800000F00706062E0CD02068006840F0010013
:102F90002168086005E02068006840F001002168B1
:102FA000086000209EE7000000000140000401408E
:102FB0000004004000080040000C004000400140B8
:102FC0000018004010B5044603492068884201D12A
:102FD000FEF7FCFE10BD00000010004010B50821F7
:102FE0000948FFF769FF0C210748FFF765FF00213B
:102FF0000548FFF761FF04210348FFF75DFF0C213F
:103000000248FFF759FF10BD840100203C01002059
:103010007047704770B50446002520684069C0F3CA
:10302000C01594F83D00212817D1B5B100BF00BFED
:103030002168143151E8001F21F08000216814310B
:1030400041E80002002AF3D100BF606B10B1606B51
:10305000FEF745FB204602F04DF820684069C0F3BA
:10306000801594F83E00222817D1B5B100BF00BFEB
:103070002168143151E8001F21F04000216814310B
:1030800041E80002002AF3D100BFA06B10B1A06B91
:10309000FEF725FB204601F0E7FF002070BD7047DA
:1030A0002DE9F84F0446206805682068C668206846
:1030B00047694FF00009CA4605F00F09B9F1000F42
:1030C0000AD105F0200038B106F0200020B12046DA
:1030D00002F023F8BDE8F88FB9F1000F7CD007F0BB
:1030E000010018B906F49070002875D005F00100B1
:1030F00030B106F4807018B1206C40F001002064FB
:1031000005F0040030B107F0010018B1206C40F068
:103110000200206405F0020030B107F0010018B190
:10312000206C40F00400206405F0080048B106F06F
:10313000200010B907F0010018B1206C40F0080021
:103140002064206C002846D005F0200028B106F04D
:10315000200010B1204601F0E0FF20684069C0F374
:10316000801A206C00F0080010B9BAF1000F2DD0C1
:10317000204601F079FF2068406900F040004028B7
:1031800020D100BF00BF2168143151E8001F21F099
:1031900040002168143141E80002002AF3D100BF49
:1031A000A06B50B17548A16B0865A06BFEF7EDFAF6
:1031B00088B1A06B016D88470DE02046FFF76FFFD7
:1031C00009E009E02046FFF76AFF04E02046FFF728
:1031D00066FF002020647DE7206B012876D105F092
:1031E0001000002872D006F010000028FAD000BFAE
:1031F00000200090206800680090206840680090DF
:1032000000BF00BF2068406900F0400040285ED148
:10321000A06B006840681FFA80F8B8F1000F54D026
:10322000A08D404551DDA4F82E80A06BC069B0F59B
:10323000807F43D000BF00BF21680C3151E8001FE0
:1032400021F4807021680C3141E80002002AF3D19A
:1032500000BF00BF00BF2168143151E8001F21F0FA
:1032600001002168143141E80002002AF3D100BFB7
:1032700000BF00BF2168143151E8001F21F0400059
:103280002168143141E80002002AF3D100BF202058
:1032900084F83E000020206300BF00BF21680C318D
:1032A00051E8001F21F0100021680C3141E80002B4
:1032B000002AF3D100BFA06BFEF711FAA08DE28DBA
:1032C000801A81B22046FFF7A4FE03E740E0A08DFC
:1032D000E18D401A1FFA80F8E08DC0B3B8F1000FFD
:1032E00035D000BF00BF21680C3151E8001F21F428
:1032F000907021680C3141E80002002AF3D100BF30
:1033000000BF00BF2168143151E8001F21F0010007
:103310002168143141E80002002AF3D100BF2020C7
:1033200084F83E000020206300BF00BF21680C31FC
:1033300051E8001F21F0100021680C3141E8000223
:10334000002AF3D100BF41462046FFF762FEC1E6E6
:1033500005F0800030B106F0800018B1204602F080
:10336000D7F8B7E605F0400030B106F0400018B1DC
:10337000204601F0AFFEADE600BFABE6354F0008DA
:1033800010B504460CB9012010BDA06900B100E0E1
:1033900000BF94F83D0028B9002084F83C00204686
:1033A00000F028F8242084F83D002068C06820F44C
:1033B00000502168C860204601F02CFF2068006999
:1033C00020F49040216808612068406920F02A00BC
:1033D000216848612068C06840F400502168C860D6
:1033E00000202064202084F83D0084F83E00002066
:1033F000CAE7000010B586B00446142101A8FCF706
:1034000089FF5F492068884259D100BF00200090A1
:103410005C48006840F010005A490860084600689F
:1034200000F01000009000BF00BF00BF002000901F
:1034300054481438006840F00100524914390860BB
:103440000846006800F00100009000BF00BF4FF484
:10345000C06001900220029000200390032004909D
:103460000720059001A94848FEF798FB47484849BE
:1034700008604FF000604860002145488160C160ED
:103480004FF4806101610021416181614FF48071DD
:10349000C161002101624162FEF7ACFA08B1FDF79B
:1034A0009DFB00BF3A48A063846300BF0022052152
:1034B0002520FEF749FD2520FEF736FD5EE0354963
:1034C000206888425AD100BF002000902D48001F7C
:1034D000006840F480202B49091F086008460068F6
:1034E00000F48020009000BF00BF00BF00200090CB
:1034F00024481438006840F002002249143908605A
:103500000846006800F00200009000BF00BF4FF4C2
:10351000406001900220029000200390032004905C
:103520000720059001A91C48FEF738FB1B481C49E1
:1035300008604FF000604860002119488160C16058
:103540004FF4806101610021416181614FF480711C
:10355000C161002101624162FEF74CFA08B1FDF73A
:103560003DFB00BF0E48A063846300BF002205211D
:103570002720FEF7E9FC2720FEF7D6FC06B010BD99
:103580000010014044380240000002404064024004
:10359000A8080020004800400004024028600240C3
:1035A0000809002070B504460D46164694F83E0002
:1035B000202816D105B10EB9012070BD00BF94F8C6
:1035C0003C00012801D10220F7E7012084F83C00EB
:1035D00000BF0020206332462946204601F030FF1C
:1035E000EBE70220E9E770477047704700BFFEE74E
:1035F00070B504460D46012C08D10C2047490860DF
:10360000C00348604FF4A00088601CE0022C07D182
:103610000C204249086080034860E004886012E0A2
:10362000032C08D103203D4908604FF40020486076
:103630002005886007E00C2038490860C003486016
:103640004FF4A00088603648364908603348006867
:103650004860002133488160C1603048416831488A
:1036600001612E4881682F48416100210176417631
:103670008176C17601774177FDF71AFE08B1FDF733
:10368000ADFA012D09D10C202449C860C10323489B
:1036900001614FF4A00141611FE0022D08D10C200F
:1036A0001E49C86081031D480161E904416114E0BD
:1036B000032D09D103201949C8604FF40021174890
:1036C00001612905416108E00C201449C860C1036B
:1036D000124801614FF4A001416113481349086089
:1036E0000E48C0684860002110488160C1600B48E6
:1036F00001690E480161094841690C484161002196
:10370000017641768176C17601774177FDF7D0FD6C
:1037100008B1FDF763FAFDF72DF870BD1801002020
:1037200000640040C800002000680040F000002055
:1037300008B500BF002000901648006840F48000E3
:10374000144908600846006800F48000009000BF3B
:1037500000BF00BF002000900846006840F4001041
:1037600008600846006800F40010009000BF00BF29
:10377000002205210C20FEF7E7FB0C20FEF7D4FB0E
:10378000002205213A20FEF7DFFB3A20FEF7CCFBB2
:1037900008BD00003038024010B50F4B0022012157
:1037A0000E4802F0FBFA0E4908600E4A00210E484E
:1037B00002F096FA0D4908600D4A00210D4802F00A
:1037C0008FFA0D4908600D4A00210D4802F088FA71
:1037D0000C49086010BD0000E0800008F5070008F3
:1037E0001000002074800008E9490008040000204F
:1037F00098800008554E000808000020BC80000892
:10380000894E00080C00002000B587B0142102A8E2
:10381000FCF780FD00BF002001903E48006840F0AA
:1038200010003C4908600846006800F01000019054
:1038300000BF00BF00BF002001900846006840F0B4
:10384000800008600846006800F08000019000BF1A
:1038500000BF00BF002001900846006840F0020051
:1038600008600846006800F00200019000BF00BF39
:1038700000BF002001900846006840F00800086082
:103880000846006800F00800019000BF00BF00BFBC
:10389000002001900846006840F04000086008469B
:1038A000006800F04000019000BF00BF00BF002092
:1038B00001900846006840F0010008600846006872
:1038C00000F00100019000BF00BF01221821124842
:1038D000FEF768FA00224FF420711048FEF762FAF2
:1038E000182002900120039000200490059002A966
:1038F0000948FEF753F94FF420700290012003901D
:1039000000200490059002A90448FEF747F907B08B
:1039100000BD000030380240001002400018024094
:1039200000B589B00020079008901C216846FCF77C
:10393000F1FC174817490860292048600021154804
:1039400081606321C160002101618161FFF765FA37
:1039500008B1FDF743F900200790089007A90D482A
:10396000FEF7F6FE08B1FDF739F96020009000205F
:103970000190029004900C2269460648FFF7CBF9AB
:1039800008B1FDF72BF90348FFF748F909B000BD6E
:10399000000400403C01002000B58DB000200990DB
:1039A0000A900B900C90079008901C216846FCF739
:1039B000B1FC2B482B490860292048600021294888
:1039C00081606321C160002101618161FEF71AFFFE
:1039D00008B1FDF703F94FF48050099009A9214877
:1039E000FEF7CAFF08B1FDF7F9F81E48FFF715FA10
:1039F00008B1FDF7F3F800200790089007A91948CF
:103A0000FEF7A6FE08B1FDF7E9F86020009000205F
:103A1000019002900490002269461248FFF77BF95A
:103A200008B1FDF7DBF8042269460E48FFF773F989
:103A300008B1FDF7D3F8082269460A48FFF76BF989
:103A400008B1FDF7CBF80C2269460648FFF763F989
:103A500008B1FDF7C3F80348FFF7E0F80DB000BD6B
:103A6000000800408401002010B513481349086085
:103A7000134848604FF48051104881604900C1608C
:103A8000C91001610C21416100218161C161FFF711
:103A900077FC08B1FDF7A2F808480068C06840F05C
:103AA000100006490968C8604FF4007205490348D0
:103AB000FFF778FD10BD0000001001402008002035
:103AC000A08601001702002010B5124812490860B4
:103AD0004FF4E130486000210F488160C16001610E
:103AE0000C21416100218161C161FFF749FC08B1EE
:103AF000FDF774F808480068C06840F010000649F7
:103B00000968C8604FF4007204490348FFF74AFD92
:103B100010BD000000480040640800201F0600207F
:103B200000BFFEE700BFFEE710B551480078C0F3C4
:103B30000010B0B94F48007890B100231A46032115
:103B40004D4801F0BBF900231A4604214A4801F010
:103B5000B5F900204949087046490870484908608D
:103B600010BD4448007898B900231A460321424802
:103B700001F0A4F92323002204213F4801F09EF91B
:103B800001203C49087003F0DBFF3D490860E7E78E
:103B90003848007801280CD103F0D2FF3849096871
:103BA000401A40F6B831884200D2D9E702203149A4
:103BB000087030480078022858D12D48007800F06D
:103BC0000100C0B92A480078C0F3400098B92B48DA
:103BD000007801280FD05A2300220321264801F043
:103BE0006DF9382300220421234801F067F90120F0
:103BF000224908703AE01E48007800F00100C0B188
:103C00001B480078C0F3400098B91C48007802288F
:103C10000FD0552300220321174801F04FF91C2330
:103C200000220421144801F049F9022013490870C8
:103C30001CE00F48007800F00100B8B90C4800788B
:103C4000C0F3400090B10D48007803280ED05F23E8
:103C500000220321084801F031F9542300220421F5
:103C6000054801F02BF903200449087000BF77E7ED
:103C700028000020210000208401002020000020D6
:103C80002400002010B51D48807801282CD1002088
:103C90001A49887008460088192806DA4FF400711E
:103CA0001648C01CFCF736FB15E000200FE0134956
:103CB000C91C0A5C12490B88091DCA54091F0988CE
:103CC000491CC1F308010E4A1180411C88B20B49FE
:103CD00009888142EBDC4FF400710848C01CFCF7F6
:103CE00019FB0020054908804FF400720349C91CE4
:103CF0000448FFF757FC02F0EBFE10BD1402002051
:103D0000B00900202008002082480089B0F58D7F8E
:103D10000CD18148007820F00100401C7E490870D9
:103D20000846007820F0020008702FE079480089EA
:103D300040F2EA3188420BD17748007820F0010048
:103D4000754908700846007820F0020008701DE0F0
:103D50007048008940F2BA6188420CD16E48007800
:103D600020F001006C4908700846007820F002003D
:103D7000801C08700AE06848007820F0010066495D
:103D800008700846007820F00200087061484089F9
:103D9000B0F58D7F0CD16048007820F00400001D44
:103DA0005D4908700846007820F0080008702FE090
:103DB0005848408940F2EA3188420BD15648007891
:103DC00020F00400544908700846007820F00800EC
:103DD00008701DE04F48408940F2BA6188420CD11A
:103DE0004D48007820F004004B49087008460078E0
:103DF00020F00800083008700AE04748007820F0FA
:103E00000400454908700846007820F00800087052
:103E100040488089B0F58D7F06D13F48007820F07A
:103E200010003D49087013E03A48808940F2BA61B9
:103E3000884207D13848007820F010001030364909
:103E4000087005E03448007820F01000324908700E
:103E50003048C089B0F58D7F06D12F48007820F01A
:103E600020002D49087013E02A48C08940F2BA6149
:103E7000884207D12848007820F0200020302649C9
:103E8000087005E02448007820F0200022490870DE
:103E90002048008AB0F58D7F06D11F48007820F0B9
:103EA00040001D49087013E01A48008A40F2BA61C8
:103EB000884207D11848007820F040004030164969
:103EC000087005E01448007820F04000124908709E
:103ED0001048408AB0F58D7F06D10F48007820F059
:103EE00080000D49087013E00A48408A40F2BA6128
:103EF000884207D10848007820F0800080300649C9
:103F0000087005E00448007820F08000024908703D
:103F100070470000061000202800002010B501F0B6
:103F200085FB10BD2DE9F04104460D46164600BF45
:103F30000E4F3878532801D001F078FB00BFEFF323
:103F400011800746202080F3118800BF00BF324651
:103F50002946204600F00CF88046F8B280F311881C
:103F600000BF00BF4046BDE8F08100000CEB002020
:103F70002DE9F047074688461646C24607EB47013B
:103F80001B4800EBC109D9F8140020B1012811D059
:103F9000022826D11EE0484601F080FB0546B542C6
:103FA00001D2002405E0344632465146484601F02D
:103FB00054FD18E0484601F071FB0546B54201D2B8
:103FC000284600E03046044622465146484601F065
:103FD00044FD08E032465146484601F003FD0446E0
:103FE00001E0002400BF00BF2046BDE8F0870000CC
:103FF00024EB00200FB438B5044606A800906A46AA
:104000002046059900F008F8054600200090284653
:1040100038BC5DF814FB00002DE9F74F2DED028B45
:1040200098B00D46144603A8139040201490002029
:1040300015901A9817900020169000BF2E786D1CCE
:1040400006B90DE1252E79D100274FF0010A00BFF6
:104050002E78232E12D02B2E0CD02D2E02D0302EC7
:1040600010D103E047F001076D1C0EE047F0020796
:104070006D1C0AE047F004076D1C06E047F00807D6
:104080006D1C02E04FF0000A00BF00BFBAF1000F44
:10409000DED14FF0000900BF2E78302E01DB392E23
:1040A00000DD07E06D1CA6F1300009EB890100EB93
:1040B0004109F1E700BF4FF000082E782E2E10D1F5
:1040C0006D1C00BF2E78302E01DB392E00DD07E09D
:1040D0006D1CA6F1300008EB880100EB4108F1E708
:1040E00000BF2E7800BF6C2E01D0682E02D16D1C4F
:1040F0002E7800E000E0F6E700BF662E73D008DC03
:10410000252E71D0582E41D0632E0BD0642E6CD149
:1041100015E0702E6BD0732E4BD0752E22D0782EDA
:10412000F5D132E02168081D2060D1F800A00AF026
:10413000FF0B594613A801F033FC86E088E02168A4
:10414000081D2060D1F800A0B8F1000F01D027F0C1
:10415000020743460A22514613A8CDE9009701F011
:1041600033FB72E02168081D2060D1F800A0B8F18F
:10417000000F01D027F0020743460A22514613A838
:10418000CDE9009701F096FB5FE000BF2168081DB4
:104190002060D1F800A0B8F1000F01D027F002078D
:1041A00043461022514613A8CDE9009701F082FB47
:1041B0004BE02168081D2060D1F800B0BBF1000F72
:1041C00001D10FF2C80B00BF9BF800600BF1010B8F
:1041D00006B906E0314613A801F0E2FB1698002864
:1041E000F2DA00BF31E017E011E02DE0FFE72168CF
:1041F000081D2060D1F800A0002008210B461022E5
:10420000CDE90010514613A801F054FB1DE0252113
:1042100013A801F0C5FB18E02068C01D20F00700BE
:1042200001460830206091ED000BB0EE408AF0EEC0
:10423000608A3B464A464146B0EE480AF0EE680ABC
:1042400013A801F039FA00E000BF00BF6D1C03E0C5
:10425000314613A801F0A4FB16980028BFF6EEAE75
:1042600000BF169800280ADD159820B103A9159AF9
:104270001A98FFF757FEDDE91510084416901698B6
:1042800018B0BDEC028BBDE8FE8F0000284E554CE7
:104290004C29000010B54448C089B0F58D7F2CD161
:1042A00041488089B0F58D7F27D13F48408940F251
:1042B000EA31884221D13C48008988421DD13B48DF
:1042C0000078D0B93848408840F28631884214DD01
:1042D0003548408840F24E4188420EDA3248008824
:1042E00040F28631884208DD2F48008840F24E4176
:1042F000884202DA01202D4908702C4800780028F5
:1043000051D0FFF701FD2A480078C0F34010002883
:1043100047D027480078C0F3800048B92448007887
:10432000C0F3C00020B94FF448702249088021E052
:104330001F480078C0F3800048B11D480078C0F3E2
:10434000C00020B94FF4FA701A49088012E01848EA
:104350000078C0F3800048B915480078C0F3C00069
:1043600020B14FF47A701349088003E04FF448708D
:104370001049088000F028F80F48B0F900300F48C5
:10438000B0F900200E48B0F900100E48B0F9000056
:10439000FCF750FAFFF7C8FB22210348FBF7BAFFEE
:1043A00001E0FCF71BFB10BD0610002029000020D7
:1043B00028000020320000202C00002030000020C7
:1043C0002A0000202E0000202DE9F0412DED048B65
:1043D0000E21FE48FBF79EFF002500260027A84679
:1043E0000024FB48408806B2F948008805B240F234
:1043F0008630854203DB40F24E40854200DD0DB938
:104400004FF0010840F28630864203DB40F24E4016
:10441000864200DD06B901277FB1B8F1000F0CD04C
:104420000020EA4988800021E848C1801020E7493F
:1044300008731021E5484173B2E20020E349087394
:104440000021E2484173002F65D1B8F1000F62D01E
:1044500040F24E4086422BDD40F2BA6086420CDBD1
:10446000DC48008800B2D9498880DA480088C04317
:10447000401C01B2D548C1806BE2A6F24E40D5493E
:10448000098848434FF41B7190FBF1F000B2CF490B
:104490008880A6F24E40CF49098848434FF41B71EB
:1044A00090FBF1F0C043401C01B2C848C18050E20B
:1044B000002EE1DD40F286308642DDDAB6F58D7FF2
:1044C0000CDCC4480088C043401C00B2BF4988804F
:1044D000C048008801B2BD48C1803AE240F286304F
:1044E000801BBC49098848434FF41B7190FBF1F0D5
:1044F000C043401C00B2B549888040F28630801B22
:10450000B449098848434FF41B7190FBF1F001B2A4
:10451000AE48C1801DE2002F7ED0B8F1000F7BD1E4
:10452000002D40DD40F2863085423CDAB5F58D7FC6
:1045300014DCA849088800EBD0716FEA6101491CBE
:1045400009B2A24A9180A349088800EBD0716FEAB2
:104550006101491C0AB29D49CA80FAE19D49088857
:1045600000EBD071491040F28632521B51434FF498
:104570001B7291FBF2F1C943491C09B2934A918025
:104580009449088800EBD071491040F28632521BE2
:1045900051434FF41B7291FBF2F1C943491C0AB21B
:1045A0008A49CA80D5E140F24E40854295DD40F20D
:1045B000BA60854210DB8749088800EBD07149104A
:1045C00009B2824A91808349088800EBD071491072
:1045D0000AB27E49CA80BCE17E49088800EBD071EE
:1045E0004910A5F24E4251434FF41B7291FBF2F178
:1045F00009B2764A91807749088800EBD07149105A
:10460000A5F24E4251434FF41B7291FBF2F10AB2F4
:104610006E49CA809DE1FFE740F24E40864260DD70
:10462000002D5EDD40F2863085425ADAA6F24E4019
:1046300040F28631491B884225DB66490988484398
:104640004FF41B7190FBF1F440F28631491B61433A
:104650004FF41B7291FBF2F0C11700EB9171A4EBC8
:10466000A10109B2594A918040F28630401B604353
:104670004FF41B7190FBF1F0201AC043401C01B2B3
:104680001046C18065E140F28630401B51490988DF
:1046900048434FF41B7190FBF1F4A6F24E42624383
:1046A0000B4692FBF3F0C21700EB92729210214678
:1046B00004EBD17302EB630212B2444B9A80A6F270
:1046C0004E4262434FF41B7392FBF3F000EBD07247
:1046D00004EBD1735B10A3EB620213B23B4AD380AD
:1046E00037E140F24E4086425ADD854258DDA6F25F
:1046F0004E40A5F24E41884221DB364909884843A5
:104700004FF41B7190FBF1F4A5F24E40604390FB17
:10471000F1F0201A00B22D498880A5F24E41614384
:104720004FF41B7291FBF2F0C11700EB9171A4EBF7
:10473000A101C943491C0AB22449CA8009E1A5F272
:104740004E402449098848434FF41B7190FBF1F413
:10475000A6F24E4262430B4692FBF3F000EBD0729E
:10476000214604EBD1735B10A3EB6202D243521CCF
:1047700012B2164B9A80A6F24E4262434FF41B735C
:1047800092FBF3F0C21700EB9272921004EBD1731C
:1047900002EB6302D243521C13B20C4AD380D8E01E
:1047A000002E72DD40F2863086426EDA002D6CDD1E
:1047B00085426ADA801B40F28631491B88422FDB32
:1047C00040F28630801B0349098805E0281000204C
:1047D000061000203200002048434FF41B7190FB6C
:1047E000F1F440F28631491B61434FF41B7291FB97
:1047F000F2F0C11700EB9171A4EBA101C943491C70
:1048000009B2714A918040F28630401B60434FF4F8
:104810001B7190FBF1F0201A01B21046C18098E0A4
:1048200040F28630401B6949098848434FF41B71A8
:1048300090FBF1F440F28632921B62430B4692FBEE
:10484000F3F0C21700EB92729210214604EBD17381
:1048500002EB6302D243521C12B25B4B9A8040F2CD
:104860008632921B62434FF41B7392FBF3F000EB12
:10487000D07204EBD1735B10A3EB6202D243521CE3
:1048800013B2514AD38064E0FFE7002E61DD40F2AD
:10489000863086425DDA40F24E40854259DD40F274
:1048A0008630811BA5F24E40814224DB40F28630E7
:1048B000801B4649098848434FF41B7190FBF1F473
:1048C000A5F24E40604390FBF1F0201AC043401C1B
:1048D00000B23D498880A5F24E4161434FF41B72FE
:1048E00091FBF2F0C11700EB9171A4EBA1010AB2A8
:1048F0003549CA802DE0A5F24E4034490988484325
:104900004FF41B7190FBF1F440F28632921B62432C
:104910000B4692FBF3F000EBD072214604EBD1730F
:104920005B10A3EB620212B2274B9A8040F28632F0
:10493000921B62434FF41B7392FBF3F0C21700EB20
:104940009272921004EBD17302EB630213B21E4A0F
:10495000D3801D49B1F90400FBF700FE41EC190BAF
:104960009FED1B0B53EC102BFBF786FD41EC180B56
:10497000FBF705FE00B214498880B1F90600FBF789
:10498000EDFD41EC190B9FED120B53EC102BFBF7D7
:1049900073FD41EC180BFBF7F2FD01B20A48C18030
:1049A000094880880C4908800748C0880B4908805E
:1049B0000548007B0A4908800348407B0949088074
:1049C000BDEC048BBDE8F0812810002032000020EF
:1049D000000000000000F03F2A0000202C00002012
:1049E0002E000020300000204FF4FA710D480068BE
:1049F00001F032FA14E008210B48FDF7C9F90B4821
:104A0000007848B10948407830B10948FDF7D6F937
:104A100000200649087048704FF4487001F00AF908
:104A2000E9E7000010000020001002400200002012
:104A30003001002010B54FF0E020006903F070F85D
:104A4000012801D002F0BAFC10BD000000B593B0FF
:104A5000302107A8FBF75EFC142102A8FBF75AFCE3
:104A600000BF002001902548006840F08050234995
:104A700008600846006800F08050019000BF00BF49
:104A800000BF002001901E48006840F480401C498F
:104A900008600846006800F48040019000BF00BF35
:104AA000092007904FF48030089001200C900220DC
:104AB0000D9041050E9104210F91A8211091022122
:104AC00011910421129107A8FDF7F2FB08B1FCF740
:104AD00085F80F20029002200390002004904FF4EC
:104AE000A05005904FF480500690052102A8FDF7D4
:104AF0007DFA08B1FCF772F813B000BD40380240EF
:104B0000007000400348006840F4700001490860EC
:104B10007047000088ED00E010B50248FDF7B3FFD4
:104B200010BD00006809002010B50268294B9842AA
:104B30000ED0B0F1804F0BD0274B984208D0274BB6
:104B4000984205D0264B984202D0264B984203D17A
:104B500022F070024B681A431E4B984220D0B0F1ED
:104B6000804F1DD01C4B98421AD01C4B984217D036
:104B70001B4B984214D01B4B984211D01A4B9842B1
:104B80000ED01A4B98420BD0194B984208D0194BB3
:104B9000984205D0184B984202D0184B984203D146
:104BA00022F44072CB681A4322F080034C6943EA36
:104BB000040202608B68C3620B688362054B9842F3
:104BC00002D0084B984201D10B6903630123436172
:104BD00010BD00000000014000040040000800403B
:104BE000000C00400004014000400140004401402E
:104BF0000048014000180040001C00400020004018
:104C000030B501F01F05012404FA05F3046A9C4342
:104C10000462046A01F01F0502FA05F52C430462E0
:104C200030BD30B50C46816821F47F4142EA03254E
:104C300025432943816030BD0A46816821F0700117
:104C400042F00703194381607047000030B5056AE0
:104C500025F001050562026A4368846924F0700446
:104C600024F003040D682C4322F002028D682A43CD
:104C7000104DA84200D103E00F4DA84206D100BF5D
:104C800022F00802CD682A4322F00402094DA8420E
:104C900002D0094DA84207D123F4807323F4007396
:104CA0004D692B438D692B43436084614D68456397
:104CB000026230BD000001400004014030B5056AC9
:104CC00025F010050562026A4368846924F4E04413
:104CD00024F440740D6844EA052422F020028D6813
:104CE00042EA0512124DA84200D103E0114DA8423C
:104CF00007D100BF22F08002CD6842EA051222F0FF
:104D000040020B4DA84202D00A4DA84209D123F41B
:104D1000806323F400634D6943EA85038D6943EAA8
:104D20008503436084614D688563026230BD000085
:104D3000000001400004014030B5056A25F480758B
:104D40000562026A4368C46924F0700424F0030415
:104D50000D682C4322F400728D6842EA0522124D40
:104D6000A84200D103E0114DA84207D100BF22F4B0
:104D70000062CD6842EA052222F480620A4DA84210
:104D800002D00A4DA84209D123F4805323F40053E2
:104D90004D6943EA05138D6943EA05134360C46115
:104DA0004D68C563026230BD00000140000401404F
:104DB00030B5056A25F480550562036A4468C26906
:104DC00022F4E04222F440720D6842EA052223F404
:104DD00000538D6843EA0533084DA84202D0084DC0
:104DE000A84204D124F480444D6944EA8514446007
:104DF000C2614D680564036230BD000000000140DF
:104E00000004014030B50B461446026A056A25F0DD
:104E100001050562816921F0F00141EA041122F0E7
:104E20000A021A438161026230BD30B50B46144656
:104E3000056A25F0100505628169026A21F4704156
:104E400041EA043122F0A00242EA031281610262C7
:104E500030BD0000002413E0FEF714FF002001F035
:104E60003DFF0546601C84B24EF66020844200DBA4
:104E70000024012003490870052000F0DBFE00BF7C
:104E8000EAE7000002000020002413E0FFF702FA26
:104E9000002001F023FF0546601C84B24EF660201E
:104EA000844200DB0024012003494870322000F0D6
:104EB000C1FE00BFEAE700000200002070B5044612
:104EC0000D460021012D06D0022D06D0032D06D05F
:104ED000042D08D105E0002007E0042005E00820AB
:104EE00003E00C2001E03C2000BF00BF632B01D990
:104EF000632103E00BB9002100E0194610B92668D0
:104F000071630BE0042802D12668B16306E008282B
:104F100002D12668F16301E02668316470BD70B586
:104F20000546284601F0A8FD044614B1D4E9001056
:104F3000884770BD70B50546AC6B0020E085E08405
:104F40002046FEF7ACF870BD70B506460025B46B80
:104F500020684069C0F3C01594F83D00212805D1B0
:104F600025B10020E084204600F0C4F820684069A4
:104F7000C0F3801594F83E00222805D125B1002009
:104F8000E085204600F070F8206C40F010002064AE
:104F90002046FEF784F870BD70B50546AC6B2868F6
:104FA000006800F48070002842D1E08500BF00BF97
:104FB00021680C3151E8001F21F4807021680C3108
:104FC00041E80002002AF3D100BF00BF00BF216802
:104FD000143151E8001F21F001002168143141E82B
:104FE0000002002AF3D100BF00BF00BF21681431C6
:104FF00051E8001F21F040002168143141E800020F
:10500000002AF3D100BF202084F83E00206B012845
:105010000ED100BF00BF21680C3151E8001F21F004
:10502000100021680C3141E80002002AF3D100BFD2
:10503000206B012804D1A18D2046FDF7EAFF02E094
:105040002046FEF7D0FA70BD70B50546AC6B206BFC
:10505000012805D1A08D41082046FDF7DAFF02E0C6
:105060002046FEF7C1FA70BD00BF00BF02680C32D7
:1050700052E8002F22F4907102680C3242E80013CB
:10508000002BF3D100BF00BF00BF0268143252E80A
:10509000002F22F001010268143242E80013002BB5
:1050A000F3D100BF016B01290ED100BF00BF026820
:1050B0000C3252E8002F22F0100102680C3242E854
:1050C0000013002BF3D100BF202180F83E100021F7
:1050D0000163704710B504462068C06820F04000A6
:1050E0002168C860202084F83D002046FEF77DFA44
:1050F000002010BD00BF00BF02680C3252E8002F34
:1051000022F0C00102680C3242E80013002BF3D1F8
:1051100000BF202180F83D107047F8B5044694F890
:105120003E00222873D1A068B0F5805F0CD12069C1
:1051300050B90025A66A20684068C0F30800308096
:10514000A06A801CA06215E0A56A0026A068B0F5E0
:10515000805F03D0A06828B9206918B9206840682A
:10516000287004E02068406800F07F002870A06A82
:10517000401CA062E08D401E80B2E085002844D132
:105180002068C06820F020002168C8602068C068DE
:1051900020F480702168C8602068406920F0010018
:1051A00021684861202084F83E00206B012826D128
:1051B0000020206300BF00BF21680C3151E8001FB0
:1051C00021F0100021680C3141E80002002AF3D1DF
:1051D00000BF2068006800F0100010280AD100BF4E
:1051E00000200090206800680090206840680090CF
:1051F00000BF00BFA18D2046FDF70BFF02E0204657
:10520000FEF7F1F90020F8BD01E00020FBE70220E5
:10521000F9E700002DE9F84F04462068006920F402
:105220004050E1680843216808612169A06808438B
:1052300061690843E169084300902068C06849F249
:105240000C618843009908432168C8602068406960
:1052500020F44070A16908432168486176492068BC
:10526000884203D075492068884203D1FCF7B8FF13
:10527000814602E0FCF7A4FF8146E069B0F5004FEB
:105280006CD102206168A0FB015003461920A9FBE4
:10529000007001462A463846FAF7F2FF6421B0FB57
:1052A000F1F04FEA001A02206168A0FB01510B46A1
:1052B0001920A9FB00712A463846FAF7E1FF834618
:1052C00002206168A0FB015003461920A9FB007170
:1052D0002A463846FAF7D4FF6421B0FBF1F000EB20
:1052E000C00101EB0010ABEB8000322101EBC000EC
:1052F0006421B0FBF1F000F0F8000AEB400A022054
:105300006168A0FB015003461920A9FB007001460B
:105310002A463846FAF7B4FF834602206168A0FBAC
:10532000015003461920A9FB00712A463846FAF7B6
:10533000A7FF6421B0FBF1F000EBC00101EB00100E
:10534000ABEB8000322101EBC0006421B0FBF1F037
:1053500000F007005044216888606AE0042061681A
:10536000A0FB015003461920A9FB007001462A4604
:105370003846FAF785FF824604206168A0FB015099
:1053800003461920A9FB007001462A463846FAF761
:1053900077FF6421B0FBF1F000EBC00101EB0010DE
:1053A000AAEB8000322101EB00106421B0FBF1F088
:1053B00000F0F00A04206168A0FB01700346192088
:1053C000A9FB00513A462846FAF75AFF6421B0FB80
:1053D000F1F00AEB001A04206168A0FB01510B46B2
:1053E0001920A9FB00712A463846FAF749FF83467F
:1053F00004206168A0FB015003461920A9FB00703E
:1054000001462A463846FAF73BFF6421B0FBF1F02B
:1054100000EBC00101EB0010ABEB8000322101EB8F
:1054200000106421B0FBF1F000F00F00504421683F
:105430008860BDE8F88F00000010014000140140B2
:1054400077B581B0044615460298A062A585002074
:105450002064222084F83E002A48A16BC8632A48B1
:10546000A16B08642948A16BC8640020A16B086582
:1054700002AE32682368191D2B46A06BFCF730FB87
:1054800000BF0020009020680068009020684068FD
:10549000009000BF00BF00BF002084F83C0000BFA8
:1054A000206970B100BF00BF21680C3151E8001FB6
:1054B00041F4807021680C3141E80002002AF3D1E8
:1054C00000BF00BF00BF2168143151E8001F41F048
:1054D00001002168143141E80002002AF3D100BF25
:1054E00000BF00BF2168143151E8001F41F04000A7
:1054F0002168143141E80002002AF3D100BF0020E6
:1055000004B070BD994F000849500008494F000889
:10551000014691F83D00212828D18868B0F5805FC8
:105520000BD1086948B90A6A1088C0F308000B68F3
:105530005860086A801C086205E00B6A581C086203
:1055400018780B685860C88C401E80B2C88458B95F
:105550000868C06820F080000B68D8600868C068E0
:1055600040F040000B68D860002070470220FCE744
:1055700038B50025114800680068C0F30015CDB1AA
:1055800000BF002000900D480068006800900B48A4
:1055900000684068009000BF00BF0848FDF73AFD72
:1055A00007480068406884B2C4F500700549088067
:1055B000012088700148FDF773FD38BD20080020E8
:1055C000A80800201402002038B500251348006800
:1055D0000068C0F30015E5B100BF002000900F483F
:1055E0000068006800900D4800684068009000BFA7
:1055F00000BF0A48FDF70EFD09480068406884B204
:10560000C4F500700749A1F808040121054880F895
:105610000A140248FDF744FD38BD0000640800206C
:10562000080900201402002000BFFEE770B5144CEA
:10563000A8212046FAF76EFE03202061606111A0C8
:10564000A0611349E1614FF4806121620021A162F0
:105650006162E1620BA020660E4961661021A166BD
:1056600000212167E1666167002505E0C5F10F00B3
:105670000949085C60556D1C102DF7D370BD000002
:105680000CEB00205465726D696E616C00000000C7
:10569000B4EB0020B4EF00202081000810B50146D3
:1056A0000A69CB689A4204D88C68641EE41AA01870
:1056B00001E0D41A601E10BD2DE9F0472DED068BD8
:1056C00082B00446B0EE409AF0EE609A0D4616465F
:1056D0001F4651EC190BFAF752FF82465046FAF773
:1056E0003DFF41EC1A0B53EC192BFAF7C2FE41ECCB
:1056F000180B9FED2F0B53EC102B51EC180BFAF7F6
:105700005DFF05D251EC180B81F0004141EC180B04
:105710009FED290B53EC102B51EC180BFAF705FEFB
:1057200041EC180B00230A2251462046CDE90067C0
:1057300000F04AF8E068002803DB2E21204600F044
:105740002FF9E06800282EDB092D00D909254FF03C
:10575000000825E09FED1A0B53EC102B51EC180BB1
:10576000FAF78AFE41EC180B51EC180BFAF707FF19
:10577000814609F13000C1B2204600F011F94846D7
:10578000FAF7ECFE41EC1A0B53EC182BFAF771FE0A
:1057900041EC180BE068002800DA03E008F101088A
:1057A000A845D7D300BF02B0BDEC068BBDE8F0879B
:1057B0000000000000000000BBBDD7D9DF7CDB3D4E
:1057C00000000000000024402DE9FC5F06460F4663
:1057D00092469846DDE90C45002F01DA784200E058
:1057E000384683464FF0010903E09BFBFAFB09F1C1
:1057F0000109D345F9DAC84500D9C14634B1002FB3
:1058000003DB05F00400042800D1641E05F002004B
:1058100010B1B8F1000F11D005F0010070B96CB1F2
:1058200008E0641E2021304600F0BAF8F068002835
:1058300000DA02E00CB1A145F3D300BFF068002804
:1058400036DB002F05DA7F422D21304600F0A8F824
:1058500007E005F00400042803D12B21304600F0B6
:105860009FF8F068002823DB05F00200022814D11D
:1058700005F0010088B9B8F1000F0ED16CB108E055
:10588000641E3021304600F08BF8F068002800DA02
:1058900002E00CB1A145F3D300BFF068002807DB9C
:1058A0004346524639463046CDE9004500F002F8FD
:1058B000BDE8FC9F2DE9FC5F8046894615461E46E3
:1058C0000C9CCDF804900127BB4605E00198B0FB85
:1058D000F5F001900BF1010B0198A842F6D25E455C
:1058E00000D9B3460D9800F00100D0B9CCB10D98A5
:1058F00000F00200022803D116B93020009001E028
:105900002020009009E0641E4046009900F048F80D
:10591000D8F80C00002800DA02E00CB1A345F2D35D
:1059200000BFD8F80C00002835DB09E0012E01D9B2
:10593000761E04E0B9FBF7FAAA4500D201E06F43F6
:10594000F4E700BF00BFB9FBF7FA0AFB1799134849
:1059500010F80A10404600F023F8D8F80C00002890
:1059600000DA03E0B7FBF5F7002FECD100BF0D988C
:1059700000F0010078B174B109E0641E20214046B6
:1059800000F00EF8D8F80C00002800DA02E00CB1A4
:10599000A345F2D300BFBDE8FC9F000031810008A1
:1059A00070B504460E46A568681C6168814206D33E
:1059B00020684655681CA060E068401CE060D4E99F
:1059C000011088420DD1A26821682069FEF7AAFA69
:1059D000A168884203D04FF0FF30E06001E0002072
:1059E000A06070BD2DE9F05F0446894617464FF070
:1059F000000AE56800BFD4F81080A84503D9A8EBD9
:105A00000500461E04E0A5EB0800401CA1680E1A24
:105A1000A068401BB04201D9304601E0A068401B9D
:105A20000646BE4201D2304600E03846064660686F
:105A300000EB050B324649465846FAF752FCB24491
:105A4000B144BF1B3544A068A84200D10025E560E1
:105A5000002FD0D15046BDE8F09F2DE9F047044615
:105A600089461546E668A068871BAF420AD9606878
:105A700000EB060A2A4649465046FAF732FC7019EE
:105A8000E06014E0B846606800EB060A424649460A
:105A90005046FAF726FCA5EB0708D4F804A009EB5A
:105AA000070142465046FAF71CFCC4F80C80BDE8DA
:105AB000F087000002480068C0F302207047000031
:105AC0000CED00E010B5002804DB0A07130E054AB0
:105AD000135406E00A07140E034A00F00F031B1FBD
:105AE000D45410BD00E400E018ED00E0EFF30580B1
:105AF000704702E008C8121F08C1002AFAD1704797
:105B00007047002001E001C1121F002AFBD170473D
:105B10002DE9F04389B007460C4615461E46DDF8D0
:105B200040804FF000092548006800F0806010B107
:105B30000120029013E02148006800F0006010B1DD
:105B4000022002900BE01D48006800F0805010B168
:105B50000420029003E0FF2009B0BDE8F08300219B
:105B60001748029A00EB021001600CB9894603E065
:105B7000012C01D14FF0040903950495CDF8149040
:105B800000200690CDF81C8002AB324603A93846AF
:105B9000FBF73CF848B10BA00BA30BA20BA10090A4
:105BA0000020FEF727FA0120D6E700BF3846FBF7B2
:105BB0003DFA0328FAD10020CEE700000864004037
:105BC000806500401B5B306D0000000020257325C0
:105BD0007343414E2073656E642074657374206452
:105BE000617461206661696C210A202573000000E0
:105BF000FEF794F9FCF7F6F8FEF728FFFDF704FE30
:105C0000FDF796FDFDF730FFFDF75EFFFDF7C4FEE3
:105C1000FDF786FE02210846FDF7EAFCFDF7DEF9F6
:105C2000FAF784FD00F016F8FDF7B6FD00F028F84D
:105C300000BFFEE770B50546FFF758FF10B16FF0E3
:105C4000050404E0002415B1284601F0CFF92046F0
:105C500070BD000010B5FFF749FF10B16FF00504EB
:105C600009E00648006820B90120044908600024C2
:105C700001E04FF0FF34204610BD000098000020E6
:105C800070B5FFF733FF10B16FF005041FE0114846
:105C90000068012819D100BF801F0021002804DB03
:105CA0000A07130E0C4A135406E00A07150E0B4A96
:105CB00000F00F031B1FD55400BF00BF0220054991
:105CC000086001F00FFA002401E04FF0FF34204695
:105CD00070BD00009800002000E400E018ED00E036
:105CE0002DE9FF4780468946144600200390FFF7C0
:105CF000FDFE00284FD1B8F1000F4CD04FF4807654
:105D000018258246471E44B3206808B1D4F800A085
:105D1000A06900B1A5692DB1382D03D8207900F014
:105D2000010018B1002004B0BDE8F087606908B137
:105D300060698608A06840B1E0685C2805D32069E6
:105D400018B1606908B1012708E0A06830B9E068BF
:105D500020B9206910B9002700E00027012F0CD1DD
:105D60002169A0684B463246CDE900510290514668
:105D7000404601F077FE03900DE067B903A8B2B288
:105D80004B465146CDE90050404601F039FE01280E
:105D900001D0002003900398C5E700002DE9FE4FD5
:105DA0000646894692461C4600200290FFF79EFE5A
:105DB00000284BD1002E49D0082000F0B7FD054641
:105DC000002D43D02E60C5F804A0B9F1000F01D119
:105DD000002700E001274FF0FF384FF0000B94B18F
:105DE000206808B1D4F800B0A06828B1E0682C2879
:105DF00002D34FF0010808E0A06830B9E06820B98C
:105E00004FF0000801E04FF00008B8F1010F0BD18E
:105E10001049A0682B463A46CDE9001001215846AA
:105E200002F071F802900BE0B8F1000F08D10948B8
:105E30002B463A4601210090584602F049F802905C
:105E4000029818B915B1284600F0F2FF0298BDE893
:105E5000FE8F00001F4F0008F8B505460E462F467E
:105E6000FFF744FE10B16FF0050411E017B96FF0B1
:105E700003040DE00020034632460421009038461A
:105E800002F0B6F8012801D1002401E06FF002040D
:105E90002046F8BD2DE9F04105460E461648076834
:105EA00016480068001D00F005FF681C38B936B1BF
:105EB00012480168091D124800F066FF1AE07C19BB
:105EC0000E4800684460BC4207D20C480168091DB6
:105ED0000C48006800F03EFF0CE008480168091D0E
:105EE0000948006800F036FF08480068844201D283
:105EF00006480460BDE8F0815C00002048000020F6
:105F000028150020500000204C00002078000020C0
:105F100010B5044600F044FF24480068401C2349A3
:105F200008602348006840B92148046008460068BA
:105F300001280DD100F02AFA0AE01E48006838B99D
:105F40001B480068C06AE16A884201D818480460AA
:105F500019480068401C18490860084600686064D9
:105F60001649E06A0968884202D91449E06A086063
:105F7000E16A01EB8101124A02EB8100211D00F070
:105F800003FF00F037FF0B48006868B1084800685D
:105F9000C06AE16A884207D24FF080500949086020
:105FA000BFF34F8FBFF36F8F10BD0000580000206C
:105FB00048000020640000207400002060000020E1
:105FC0007810002004ED00E008B500F0E9FE12486A
:105FD0000068E8B9114800F0ADFE114800F0AAFED3
:105FE0000E48104908600E480F49086000200F4B0A
:105FF0000F4A102100900A2001F0FAF906490860C2
:106000000846006820B10BA10348006800F0B2FF09
:1060100000F0F0FE08BD00008C0000203C150020C0
:106020005015002084000020880000206415002006
:10603000B4150020546D72510000000010B516E038
:1060400000F0AEFE0C48C068C468201D00F032FEAF
:106050000A480068401E0949086009480068401E57
:106060000749086000F0C6FE204600F05FF80448CB
:1060700000680028E4D110BD14150020580000204D
:106080005400002070B504460D46206C70B1216CA0
:10609000E0680144E160D4E90210884201D321683C
:1060A000E1602846226CE168FAF71BF970BD2DE922
:1060B000F04104460F4615464FF00008A66B206CD1
:1060C00048B9206800282CD1A06801F0E1FD804685
:1060D0000020A06025E07DB93946226C6068FAF79F
:1060E00000F9216C606808446060D4E901018842CD
:1060F00017D32068606014E03946226CE068FAF734
:10610000F0F8216CE068411AE1602168E06888429B
:1061100003D2216CA068411AE160022D01D106B1C1
:10612000761E701CA0634046BDE8F08110B50446A1
:1061300094F8590030B9206B00F07AFE204600F048
:1061400077FE1AE094F85900012803D1204600F0A8
:106150006FFE12E094F85900022801D1012000E0FE
:10616000002050B900BF502080F31188BFF34F8F3B
:10617000BFF36F8F00BF00BFFEE710BD0146084AA6
:10618000126812680AB9012200E000220A600A6857
:1061900022B9034A1268D268106800E000207047F4
:1061A0008400002030B54FF44843174800F007043E
:1061B0002CB1C01D20F00700134C041B1B1B024612
:1061C000124C22600024114D6C60D018083820F069
:1061D00007000F4C206000240D4D2D686C600C4DA5
:1061E0002D682C601146441A4C60094C24680C60E0
:1061F000084D4C682C60084D4C682C604FF00044F2
:10620000064D2C6030BD00000C2300209C000020B7
:10621000A4000020AC000020A8000020B80000204E
:1062200000BFFFF70BFF064800680128F9D94FF0BF
:10623000805004490860BFF34F8FBFF36F8FF0E7C2
:106240007810002004ED00E02DE9F04106460D46EF
:1062500017469846069C0DB9246000E02760E66367
:1062600025640121204601F033F984F84C80BDE813
:10627000F0812DE9F05F82460E4690469B460A9FCC
:106280000C9C4FEA8801A522206BFAF73CF8A8F194
:106290000100216B01EB800929F0070909F00700D3
:1062A00008B9012000E0002050B900BF502080F361
:1062B0001188BFF34F8FBFF36F8F00BF00BFFEE7A2
:1062C00086B1002507E0715D04F134004155705D31
:1062D00000B902E06D1C102DF5D300BF0021432052
:1062E000015502E0002084F83400382F00D337270E
:1062F000E762E76400202065201D00F028FD04F11E
:10630000180000F024FD2461C7F13800A061646228
:106310000020606584F858005A465146484600F00F
:10632000C1FB20600B9808B10B980460BDE8F09F9A
:106330002DE9F04706460D4617469846DDE90894D4
:106340000DB1012000E0002050B900BF502080F3C3
:106350001188BFF34F8FBFF36F8F00BF00BFFEE701
:106360008CB1FFF731FE2660A561C4F81C80C4F82B
:106370002090201D00F0EBFC2FB194F8280040F095
:10638000040084F82800BDE8F087000010B5002460
:1063900007E004EB84010F4A02EB810000F0CAFC25
:1063A000641C382CF5D30C4800F0C4FC0B4800F0FA
:1063B000C1FC0B4800F0BEFC0A4800F0BBFC0A48D8
:1063C00000F0B8FC0448094908600448084908601E
:1063D00010BD000078100020D8140020EC1400201C
:1063E0000015002014150020281500204C00002066
:1063F0005000002010B50146164800E00068036810
:106400008B42FBD30246436813448B4204D143685A
:106410004C682344436001460A464B6813440468B1
:10642000A34211D10C4C03682468A34208D04B68E6
:106430000468646823444B6003681B680B6005E0D4
:10644000054B1B680B6001E003680B60884200D0BD
:10645000016010BD9C000020A40000202DE9F04147
:1064600004460D4616461F464FF00008656024613D
:10647000B5420CD8F01BA169884202D34FF0010845
:1064800011E0211D0948006800F064FC0BE0BE42E9
:1064900004D2BD4202D34FF0010804E0211D04489C
:1064A000006800F057FC4046BDE8F08188000020FD
:1064B0008400002070B5054600F072FCA86B08B996
:1064C000012400E0002400F095FC204670BD70B56A
:1064D000054600F065FCA86BE96B884201D10124F8
:1064E00000E0002400F086FC204670BDF8B50546AB
:1064F0000F461A480068C068C468201D00F0DAFB27
:1065000094F8280000F00400E8B1A06941192B4676
:106510003A462046FFF7A2FFD8B1002003462A469C
:1065200001460090204601F063FD064656B900BFC3
:10653000502080F31188BFF34F8FBFF36F8F00BFE0
:1065400000BFFEE705E094F8280020F0010084F881
:1065500028002046216A8847F8BD000084000020FA
:10656000F0B587B0A0E00398002811DA04AE56B960
:1065700000BF502080F31188BFF34F8FBFF36F8FA0
:1065800000BF00BFFEE7D6E90020B168904700BF1A
:1065900003980028E6DB059C606908B9012000E04B
:1065A000002010B9201D00F085FB02A800F0DEF8E5
:1065B000054603980A2875D2DFE800F00905073977
:1065C000416306083A4200BF00BF00BF00BF94F815
:1065D000280040F0010084F828000498A26981187E
:1065E00003462A462046FFF739FFF8B12046216AC4
:1065F000884794F8280000F00400B8B1002000900B
:106600000498A169421800231946204601F0F0FCC5
:10661000074657B900BF502080F31188BFF34F8F52
:10662000BFF36F8F00BF00BFFEE700BF3BE000BFBE
:1066300094F8280020F0010084F8280033E000BF1F
:1066400094F8280040F0010084F828000498A06124
:10665000A06908B1012000E0002050B900BF50201F
:1066600080F31188BFF34F8FBFF36F8F00BF00BF60
:10667000FEE7A06941192B462A462046FFF7EEFEA9
:1066800011E094F8280000F0020018B9204600F04C
:10669000CFFB05E094F8280020F0010084F82800E2
:1066A00001E0FFE700BF00BF002203A90448006823
:1066B00001F0ACF800287FF456AF07B0F0BD000041
:1066C0008C000020F8B505460C4600F067FD6846D2
:1066D00000F04CF80646009820BB44B9B54206D8F5
:1066E00001F074FB31462846FFF700FF1CE03CB187
:1066F0000E480068006808B9012000E00020044648
:10670000A91B22460A48006800F04AFC01F05EFB23
:1067100050B94FF0805007490860BFF34F8FBFF367
:106720006F8F01E001F052FBF8BD000088000020EF
:106730008C00002004ED00E00A490968096809B9E5
:10674000012100E0002121B14FF0FF31064A116024
:1067500006E004490968C968C868034A41681160CD
:10676000704700004C0000207800002070B50446FF
:1067700001F0E6F9054607480068854204D200F0BA
:106780000BF80120206001E0002020600148056036
:10679000284670BD940000202DE9F84334E02548D8
:1067A0000068C068056823480068C068C468201D88
:1067B00000F080FA2046216A884794F8280000F00B
:1067C000040008B3A0694619AE4207D96660246187
:1067D000211D1848006800F0BDFA15E000200346AE
:1067E0002A4601460090204601F002FC074657B9B0
:1067F00000BF502080F31188BFF34F8FBFF36F8F1E
:1068000000BF00BFFEE700BF0A480068006808B983
:10681000012000E000200028C1D00648D0F8008008
:1068200005480068034908600348C0F80080BDE8D7
:10683000F883000084000020880000200246002128
:1068400001E0521C491C1078A528FAD0890888B2AA
:10685000704700000E480068401C08B9012000E0A5
:10686000002050B900BF502080F31188BFF34F8F34
:10687000BFF36F8F00BF00BFFEE700BF502080F363
:106880001188BFF34F8FBFF36F8F00BF00BFFEE7CC
:10689000BC00002008B500BF6846FFF76FFC044647
:1068A00020460099FFF70EFFFFF75AFEF4E770B598
:1068B000044600F075FA94F9455010E0606A08B992
:1068C000012000E0002038B904F1240001F032FA80
:1068D00018B100F0C5FB00E003E0681E45B2002DD2
:1068E000ECDC00BFFF2084F8450000F083FA00F0E4
:1068F00057FA94F9445010E0206908B9012000E0EB
:10690000002048B904F1100001F014FA08B100F0B9
:10691000A7FB681E45B200E001E0002DECDC00BFE3
:10692000FF2084F8440000F065FA70BD2DE9F041C5
:1069300004464FF0000800F031FC4948006808B9EF
:10694000FFF730FC474800682040002870D1D4B1E0
:10695000083404F00700B0B104F00700C0F10800EB
:10696000044404F0070008B9012000E0002050B9F9
:1069700000BF502080F31188BFF34F8FBFF36F8F9C
:1069800000BF00BFFEE7002C52D0374800688442A9
:106990004ED8364E3046056801E02E462D686868B0
:1069A000A04202D228680028F7D12D48006885420D
:1069B0003ED0306800F10808286830606868001B25
:1069C000102819D92F1907F0070008B9012000E095
:1069D000002050B900BF502080F31188BFF34F8FC3
:1069E000BFF36F8F00BF00BFFEE76868001B7860D1
:1069F0006C603846FFF7FEFC1B4968680968081A96
:106A0000194908600846006819490968884203D294
:106A10001548006816490860124968680968084303
:106A200068600020286013480068401C1149086015
:106A300001F0CCF908F0070008B9012000E00020BF
:106A400050B900BF502080F31188BFF34F8FBFF3C0
:106A50006F8F00BF00BFFEE74046BDE8F081000039
:106A6000A4000020B8000020A80000209C00002006
:106A7000AC000020B000002070B50446254654B993
:106A800000BF502080F31188BFF34F8FBFF36F8F8B
:106A900000BF00BFFEE700F083F9EE6900F0AAF93D
:106AA000304670BD001F4FF080730360001F21F05F
:106AB00001030360001F054B036014380260001FD0
:106AC0006FF002030360203870470000556800082B
:106AD00010B52948008828494988884200D110BD4E
:106AE00025484188001D405C0F283BD12248408842
:106AF0001830C0F308012048001D405C88BB1E48C8
:106B000040881730C0F308011B48001D405C40BBA3
:106B10001948008818494988401AC0F30800192804
:106B200027DB00240BE0144840882044C0F3080110
:106B30001148001D405C11490855601CC4B2192C55
:106B4000F1DB0E4800F01CF8FDF7DEF80A4840883B
:106B50001930C0F30800084948800020A1F8060257
:106B600007E0FFE704484088401CC0F308000249E2
:106B7000488000BFB3E70000B0090020EC0F002000
:106B80004178827841EA0221C1F30A01484A118022
:106B90008178C910C27841EA4211C1F30A01444A1E
:106BA0005180C1788911027941EA8201427941EA32
:106BB0008221C1F30A013E4A9180417949108279CC
:106BC00041EAC211C1F30A01394AD1808179091120
:106BD000C27941EA0211C1F30A01354A1181C17932
:106BE000C911027A41EA4201427A41EA4221C1F3E3
:106BF0000A012F4A5181417A8910827A41EA821131
:106C0000C1F30A012A4A9181817A4911C27A41EA83
:106C1000C201274AD181017B427B41EA0221C1F3B3
:106C20000A01234A1182417BC910827B41EA421149
:106C3000C1F30A011E4A5182817B8911C27B41EA5C
:106C40008201027C41EA8221C1F30A01184A918241
:106C5000017C4910427C41EAC211C1F30A01144A85
:106C6000D182417C0911827C41EA0211C1F30A01FF
:106C70000F4A1183817CC911C27C41EA4201027D25
:106C800041EA4221C1F30A01094A5183017D891079
:106C9000427D41EA8211C1F30A01054A9183417D97
:106CA0004911827D41EAC201014AD1837047000047
:106CB0000610002001460A69D1E901309860D1E947
:106CC000010358605068884201D1886850600020F4
:106CD00008611068401E1060106870472DE9F0418F
:106CE000044614B90648006800E0204607463D6B9C
:106CF0002846FFF7A3FD06463046BDE8F0810000B8
:106D000048000020034B0360034B0B604FF480737B
:106D10001360704754160020B0160020034B036028
:106D2000034B0B604FF4007313607047B01A0020E0
:106D30000C1B002000F1080141604FF0FF31816021
:106D400000F10801C160016100210160704700216C
:106D50000161704710B502460B685C1C0CB91069E4
:106D600007E002F1080000E04068446824689C42A3
:106D7000FAD944684C604C68A160886041600A613F
:106D80001468641C146010BD42684A6093688B608C
:106D9000936859609160086103685B1C03607047E9
:106DA00000BF502080F31188BFF34F8FBFF36F8F68
:106DB00000BF0E480068401C0C4908600846006887
:106DC000012812D10A480068C0B208B9012000E0C9
:106DD000002050B900BF502080F31188BFF34F8FBF
:106DE000BFF36F8F00BF00BFFEE77047BC000020FD
:106DF00004ED00E00D48006850B900BF502080F35A
:106E00001188BFF34F8FBFF36F8F00BF00BFFEE746
:106E100006480068401E054908600846006820B919
:106E2000002080F3118800BF00BF7047BC00002025
:106E300070B506463546002E44D0083D2C46224902
:106E400060680968084008B1012000E0002050B9DE
:106E500000BF502080F31188BFF34F8FBFF36F8FB7
:106E600000BF00BFFEE7206808B9012000E0002055
:106E700050B900BF502080F31188BFF34F8FBFF38C
:106E80006F8F00BF00BFFEE70F49606809680840C8
:106E9000C0B12068B0B90C49606809688843606077
:106EA00000F07CF9094960680968084407490860EE
:106EB0002046FFF79FFA06480068401C0449086016
:106EC00000F084FF70BD0000B8000020A800002082
:106ED000B400002000204FF0E021086188610648DE
:106EE00000684FF47A71B0FBF1F0401E4FF0E021E2
:106EF00048610720086170474400002070B5F9F729
:106F0000A9F90446102C16D304F1E02090F8F053B0
:106F100015480078854201DB012000E0002050B9CF
:106F200000BF502080F31188BFF34F8FBFF36F8FE6
:106F300000BF00BFFEE70D48006800F4E0600C49A8
:106F40000968884201D8012000E0002050B900BF44
:106F5000502080F31188BFF34F8FBFF36F8F00BFB6
:106F600000BFFEE770BD0000C00000200CED00E097
:106F7000C4000020024600200BE0084B53F83030DC
:106F800033B9064B43F8301003EBC0035A6002E0FC
:106F9000401C0828F1D300BF7047000038100020C3
:106FA0002DE9F04105460E4617462C46FFF7F8FE40
:106FB00094F94400401C10B9002084F8440094F96E
:106FC0004500401C10B9002084F84500FFF712FF6F
:106FD000A06B28B93A46314604F1240000F062F86B
:106FE0002046FFF764FCBDE8F081000070B5044660
:106FF0000025D4B11248006808B9012000E0002043
:1070000050B900BF502080F31188BFF34F8FBFF3FA
:107010006F8F00BF00BFFEE700F0C0F800212046E0
:10702000FEF738FF00F0D2FE05463DB94FF0805024
:1070300004490860BFF34F8FBFF36F8F70BD00002E
:107040008000002004ED00E0034909680160034965
:107050000968416070470000700000205C0000205B
:1070600001200149086070476C00002070B504469B
:107070000D4654B900BF502080F31188BFF34F8FE5
:10708000BFF36F8F00BF00BFFEE7054801681831EE
:107090002046FFF75FFE01212846FEF7FBFE70BD8C
:1070A0004800002070B505460E46144655B900BF8D
:1070B000502080F31188BFF34F8FBFF36F8F00BF55
:1070C00000BFFEE70648016818312846FFF75CFE5E
:1070D0000CB14FF0FF3621463046FEF7DBFE70BDA7
:1070E0004800002010B586B000200590049003AA47
:1070F00004A905A8FFF706FE0022DDE904101346E7
:10710000CDE9002102901EA11F48039A00F0AAFCBD
:107110001E4908600846006808B1012400E0002408
:10712000012C02D100F028FF0446012C15D100BF2C
:10713000502080F31188BFF34F8FBFF36F8F00BFD4
:107140004FF0FF301249086001201249086000200A
:107150001149086000F07EF810E0601C08B10120C1
:1071600000E0002050B900BF502080F31188BFF329
:107170004F8FBFF36F8F00BF00BFFEE706B010BD9B
:1071800049444C4500000000216200087C000020BA
:1071900078000020640000205C00002002480068A5
:1071A000401C014908607047800000201E480068AC
:1071B00018B101201D49086034E000201B49086017
:1071C0001B4801680CE051B900BF502080F31188C2
:1071D000BFF34F8FBFF36F8F00BF00BFFEE7491EA5
:1071E00001EB8100134A52F8200008B9012000E0A9
:1071F00000200028E7D101EB81020E4B03EB820057
:1072000042685268426000F108024368934202D12A
:107210004268526842604268D268074B1A6004486C
:10722000016000BF70470000800000206C0000205B
:10723000600000207810002048000020014800680D
:1072400070470000A8000020014800687047000057
:10725000AC0000201CB5524800685249884201D059
:10726000012000E0002050B900BF502080F31188B9
:10727000BFF34F8FBFF36F8F00BF00BFFEE74848DB
:1072800000684849491E884201D0012000E00020E2
:1072900050B900BF502080F31188BFF34F8FBFF368
:1072A0006F8F00BF00BFFEE73F490846007801909E
:1072B000FF200A4610700846007800909DF80000F4
:1072C00000F0F0009DF80020904201D1012000E084
:1072D000002050B900BF502080F31188BFF34F8FBA
:1072E000BFF36F8F00BF00BFFEE79DF8000000F006
:1072F00050002E4A107007202D4A106009E02C48DB
:107300000068401E2A4A10609DF800004006000EEA
:1073100000909DF8000000F080008028EFD0244805
:107320000068C0F10700042801D1012000E000201E
:1073300050B900BF502080F31188BFF34F8FBFF3C7
:107340006F8F00BF00BFFEE7194800680002184AAF
:1073500010601046008800F4E0601060124A019846
:1073600010700F482030006840F470000C49203144
:1073700008600846006840F070400860FFF7AAFD0A
:1073800000200C490860F8F72DFF0B48006840F01A
:10739000404009490860F8F711FF00201CBD0000BB
:1073A00000ED00E071C20F4100E400E0C0000020E9
:1073B000C4000020BC00002034EF00E010B500BF86
:1073C000502080F31188BFF34F8FBFF36F8F00BF42
:1073D00000F0BCFB18B14FF080500449086000BFBA
:1073E000002080F3118800BF10BD000004ED00E014
:1073F0002DE9F84380460E4617461D46DDF82090DD
:10740000B8F1000F01D0012000E0002050B900BF0A
:10741000502080F31188BFF34F8FBFF36F8F00BFF1
:1074200000BFFEE70DB1012000E0002050B900BF11
:10743000502080F31188BFF34F8FBFF36F8F00BFD1
:1074400000BFFEE707B10EB1012000E0002050B9F7
:1074500000BF502080F31188BFF34F8FBFF36F8FB1
:1074600000BF00BFFEE707B90EB9012000E0002011
:1074700050B900BF502080F31188BFF34F8FBFF386
:107480006F8F00BF00BFFEE750200090009850288B
:1074900001D1012000E0002050B900BF502080F34E
:1074A0001188BFF34F8FBFF36F8F00BF00BFFEE7A0
:1074B00000BF2C464CB1012084F846004B463A46AA
:1074C000314640460094FEF7BFFE2046BDE8F883F3
:1074D00070B505460E462C4654B900BF502080F3C7
:1074E0001188BFF34F8FBFF36F8F00BF00BFFEE760
:1074F000FFF756FCD4E90F12206801FB0200A060E0
:107500000020A06320686060E06B401E226C216850
:1075100000FB0211E160FF2084F8440084F845007C
:107520009EB9206908B9012000E00020A8B904F143
:10753000100000F0FFFB80B14FF080500949086057
:10754000BFF34F8FBFF36F8F07E004F11000FFF719
:10755000F1FB04F12400FFF7EDFBFFF74BFC0120EA
:1075600070BD000004ED00E02DE9FF4383B0064646
:1075700088461D464FF00009344654B900BF5020DC
:1075800080F31188BFF34F8FBFF36F8F00BF00BF31
:10759000FEE7B8F1000F01D1206C08B9012000E02E
:1075A000002050B900BF502080F31188BFF34F8FE7
:1075B000BFF36F8F00BF00BFFEE7022D02D1E06B6B
:1075C000012801D1012000E0002050B900BF502067
:1075D00080F31188BFF34F8FBFF36F8F00BF00BFE1
:1075E000FEE700F09DFA08B9059808B9012000E00F
:1075F000002050B900BF502080F31188BFF34F8F97
:10760000BFF36F8F00BF00BFFEE700BFFFF7C8FBEF
:10761000A06BE16B884201D3022D28D12A46414656
:107620002046FEF744FD0746606A08B9012000E0E5
:10763000002068B904F1240000F07CFB88B14FF011
:10764000805032490860BFF34F8FBFF36F8F08E05F
:107650003FB14FF080502D490860BFF34F8FBFF30B
:107660006F8FFFF7C7FB012007B0BDE8F0830598D7
:1076700018B9FFF7BFFB0020F6E7B9F1000F04D1FE
:1076800001A8FFF7E1FC4FF00109FFF7B3FBFFF79B
:1076900085FDFFF785FB94F94400401C10B90020DC
:1076A00084F8440094F94500401C10B9002084F887
:1076B0004500FFF79FFB05A901A800F05BF9F0B9B1
:1076C0002046FEF704FFA0B104F110000599FFF772
:1076D000CDFC2046FFF7EBF800F078FB002895D1B1
:1076E0004FF0805009490860BFF34F8FBFF36F8F91
:1076F0008CE72046FFF7DBF800F068FB86E72046C2
:10770000FFF7D5F800F062FB0020ADE704ED00E0E4
:107710002DE9F84F07468A4690461E463C4654B926
:1077200000BF502080F31188BFF34F8FBFF36F8FDE
:1077300000BF00BFFEE7BAF1000F01D1206C08B90D
:10774000012000E0002050B900BF502080F31188D4
:10775000BFF34F8FBFF36F8F00BF00BFFEE7022E56
:1077600002D1E06B012801D1012000E0002050B9D6
:1077700000BF502080F31188BFF34F8FBFF36F8F8E
:1077800000BF00BFFEE7FFF7B9FB00BF5021EFF3DA
:10779000118081F31188BFF34F8FBFF36F8F00BF4C
:1077A0000546A06BE16B884201D3022E25D194F9E6
:1077B00045B0A06B0090324651462046FEF777FC5C
:1077C0000BF1010088B9606A08B9012000E00020CF
:1077D00050B904F1240000F0ADFA28B1B8F1000F5F
:1077E00002D00120C8F8000004E00BF1010040B213
:1077F00084F845004FF0010901E04FF0000900BF97
:1078000085F3118800BF4846BDE8F88F2DE9F741A0
:1078100083B005460E464FF000082C4654B900BF11
:10782000502080F31188BFF34F8FBFF36F8F00BFDD
:1078300000BFFEE70EB9206C08B9012000E000206F
:1078400050B900BF502080F31188BFF34F8FBFF3B2
:107850006F8F00BF00BFFEE700F062F908B905981E
:1078600008B9012000E0002050B900BF502080F38B
:107870001188BFF34F8FBFF36F8F00BF00BFFEE7CC
:1078800000BFFFF78DFAA76BF7B131462046FEF730
:10789000F9FB781EA063206908B9012000E00020F0
:1078A00060B904F1100000F045FA38B14FF0805093
:1078B0002F490860BFF34F8FBFF36F8FFFF79AFA1E
:1078C000012006B0BDE8F081059818B9FFF792FADB
:1078D0000020F6E7B8F1000F04D101A8FFF7B4FBD0
:1078E0004FF00108FFF786FAFFF758FCFFF758FA48
:1078F00094F94400401C10B9002084F8440094F925
:107900004500401C10B9002084F84500FFF772FACA
:1079100005A901A800F02EF8F0B92046FEF7CAFD2F
:10792000A0B104F124000599FFF7A0FB2046FEF763
:10793000BEFF00F04BFA0028A3D14FF080500C4955
:107940000860BFF34F8FBFF36F8F9AE72046FEF7B3
:10795000AEFF00F03BFA94E72046FEF7A8FF00F0E8
:1079600035FA2046FEF7A6FD00288AD00020A8E7B9
:1079700004ED00E070B505460C4655B900BF502037
:1079800080F31188BFF34F8FBFF36F8F00BF00BF2D
:10799000FEE754B900BF502080F31188BFF34F8F2A
:1079A000BFF36F8F00BF00BFFEE7FFF7F9F9124882
:1079B00002686868131A2068401C08B9002617E09E
:1079C0000E4928680968884204D06868904201D846
:1079D00001260DE02068984207D92068C01A20606F
:1079E0002846FFF731FB002602E000202060012638
:1079F000FFF700FA304670BD5C00002070000020E8
:107A00002DE9FF4F85B0804689461746DDE912AB68
:107A1000B800FEF78BFF064656B15C20FEF786FFE6
:107A200004460CB1266304E03046FFF701FA00E09B
:107A300000248CB1002084F85900CDE900ABCDE9D9
:107A400002403A4649464046089BFEF712FC204653
:107A5000FEF75EFA012501E04FF0FF35284609B038
:107A6000BDE8F08F2DE9F04F85B007468846914676
:107A70009A46DDE90EB6109C0EB1012000E0002010
:107A800050B900BF502080F31188BFF34F8FBFF370
:107A90006F8F00BF00BFFEE70CB1012000E00020A7
:107AA00050B900BF502080F31188BFF34F8FBFF350
:107AB0006F8F00BF00BFFEE75C20039003985C2837
:107AC00001D1012000E0002050B900BF502080F318
:107AD0001188BFF34F8FBFF36F8F00BF00BFFEE76A
:107AE00000BFB4B1AEB125462C462E63022085F806
:107AF0005900002004A953464A46CDE900B1CDE91A
:107B0000025041463846FEF7B4FB2846FEF700FA1D
:107B100001E000200490049805B0BDE8F08F00005B
:107B20000549096809B9012005E00449096809B94E
:107B3000022000E000207047640000208000002048
:107B400001490868704700005C0000202DE9F04101
:107B50004FF000084348006800287BD14248006885
:107B6000451C4148056015BB40480068006808B9DD
:107B7000012000E0002050B900BF502080F31188A0
:107B8000BFF34F8FBFF36F8F00BF00BFFEE73748D3
:107B90000768374800683549086035480760354848
:107BA0000068401C33490860FEF7C6FD00BF32483C
:107BB000006885423BD300BF2C480068006808B9C4
:107BC000012000E0002020B14FF0FF302A4908607A
:107BD0002CE026480068C068C4686668B54202D2D6
:107BE0002548066022E0201DFFF764F8A06A18B15E
:107BF00004F11800FFF75EF82049E06A096888423E
:107C000002D91E49E06A0860E16A01EB81011C4A61
:107C100002EB8100211DFFF7B7F81A49E06A0968F5
:107C2000C96A8842C8D34FF00108C5E700BF1548AC
:107C30000068C06A00EB8000114951F8200001285B
:107C400001D94FF001081048006808B14FF0010851
:107C500005E0FFE70D480068401C0C4908604046FD
:107C6000BDE8F081800000205C0000204C00002076
:107C700050000020700000207800002060000020EC
:107C800078100020480000206C00002068000020D0
:107C900070B505462C460026002D43D022480068CA
:107CA000844201D1012000E0002050B900BF5020E3
:107CB00080F31188BFF34F8FBFF36F8F00BF00BFFA
:107CC000FEE7206D50B900BF502080F31188BFF34C
:107CD0004F8FBFF36F8F00BF00BFFEE7206D401EC8
:107CE0002065E16CE06A88421CD0206DD0B9201D6F
:107CF000FEF7E0FFE06CE062E06AC0F13800A061EE
:107D00000A49E06A0968884202D90849E06A0860BD
:107D1000E16A01EB8101064A02EB8100211DFFF7B8
:107D200033F80126304670BD480000206000002076
:107D30007810002070B50646F068C46854B900BFDA
:107D4000502080F31188BFF34F8FBFF36F8F00BFB8
:107D500000BFFEE704F11800FEF7ACFF154800680D
:107D6000A0B9201DFEF7A6FF1349E06A0968884202
:107D700002D91149E06A0860E16A01EB81010F4A0A
:107D800002EB8100211DFEF7FFFF04E004F1180162
:107D90000B48FEF7F9FF0B49E06A0968C96A884297
:107DA00004D9012501200849086000E00025284683
:107DB00070BD0000800000206000002078100020CE
:107DC00000150020480000206C00002070B5002441
:107DD00000263648006850B900BF502080F3118853
:107DE000BFF34F8FBFF36F8F00BF00BFFEE7FEF7FB
:107DF000D7FF2E480068401E2C49086008460068DE
:107E000000284ED12A48006800284AD023E029489B
:107E1000C068C46804F11800FEF74CFF201DFEF78F
:107E200049FF2549E06A0968884202D92249E06A87
:107E30000860E16A01EB8101204A02EB8100211D0B
:107E4000FEF7A2FF1E49E06A0968C96A884202D3A8
:107E500001201C4908601748006808B9012000E0AB
:107E600000200028D3D00CB1FEF766FC1648056848
:107E700065B100BFFFF76AFE10B10120114908602B
:107E80006D1E002DF6D100200F4908600D480068D6
:107E900038B1012630070D490860BFF34F8FBFF39B
:107EA0006F8FFEF7A7FF304670BD000080000020F6
:107EB00058000020001500206000002078100020ED
:107EC000480000206C0000206800002004ED00E065
:107ED0002DE9FC4705460E4617469846DDF82890E2
:107EE0002C20FEF723FD044654B1002084F828001E
:107EF00043463A4631462846CDE90094FEF718FA43
:107F00002046BDE8FC872DE9FC4706460F46904613
:107F10009946DDE90AA52C20019001982C2801D171
:107F2000012000E0002050B900BF502080F31188EC
:107F3000BFF34F8FBFF36F8F00BF00BFFEE700BFDF
:107F400055B900BF502080F31188BFF34F8FBFF3A6
:107F50006F8F00BF00BFFEE72C4654B1022084F8AB
:107F600028004B46424639463046CDE900A4FEF78C
:107F7000DFF92046BDE8FC8710B586B00024FEF787
:107F800023F816480068D0B100200590049003AA99
:107F900004A905A8FEF7C2FE0222DDE904100023B1
:107FA000CDE9002102900EA10F48039AFFF75AFD78
:107FB0000E4908600846006800B1012400BF54B9AA
:107FC00000BF502080F31188BFF34F8FBFF36F8F36
:107FD00000BF00BFFEE7204606B010BD8C000020A9
:107FE000546D72205376630095680008900000205D
:107FF0002DE9FF4704460D4616461F46DDF8308042
:108000004FF0000954B900BF502080F31188BFF32E
:108010004F8FBFF36F8F00BF00BFFEE714480068AB
:1080200010B3009501960294062D15DAFFF778FD3E
:10803000022808D10023424669460D480068FFF730
:1080400093FA814610E000231A4669460848006802
:10805000FFF78AFA814607E000233A46694604485A
:108060000068FFF755FB8146484604B0BDE8F0873D
:108070008C00002068810008000000000000000063
:1080800000000000000000000008000028000000C0
:108090000000000000000000508100080000000007
:1080A00000000000000000000000000000080000C8
:1080B0002000000000000000000000005C810008BB
:1080C00000000000000000000000000000000000B0
:1080D0000008000010000000000000000000000088
:1080E00044810008000000000000000000000000C3
:1080F0000006101600061016000000000000000028
:10810000010203040607080900000000010203043D
:1081100030313233343536373839414243444546BD
:108120000000000000005454522052454747455378
:1081300000303132333435363738394142434445E3
:10814000460000006D7954696D65723031000000A1
:108150006D795461736B3032000000006D795461A9
:10816000736B30330000000064656661756C745495
:1081700061736B009481000800000020C8000000BB
:10818000F25A00085C820008C800002000F30000DA
:10819000025B00080000000000000000000000007A
:1081A00000000000000000000000000000000000CF
:1081B00000000000000000000000000000000000BF
:1081C000000000000000F4010000000000000000BA
:1081D00010000000010000000024F4000000000076
:1081E000000000000000000000000000000000008F
:1081F000000000000000000000000000000000007F
:10820000000000000000000000000000000000006E
:10821000000000000000000000000000000000005E
:10822000000000000000000000000000000000004E
:10823000000000000000000000000000000000003E
:10824000000000000000000000000000000000002E
:0C825000AAAAAAAA00000000000000007A
:040000050800018965
:00000001FF
